S01C00006376615F626F6F746C6F616465725F6D303131382E73726563AE
S1130000F05B002071C100009B2D00000B4000003C
S113001000000000000000000000000000000000DC
S11300200000000000000000000000006741000024
S1130030000000000000000067420000B35C000004
S113004004C5000004C5000004C5000004C5000088
S113005004C5000004C5000004C5000004C5000078
S113006004C50000D55C000004C5000004C5000000
S113007004C5000004C5000004C5000004C5000058
S113008004C5000004C5000004C5000004C5000048
S113009004C5000004C5000004C5000004C5000038
S11300A0BD64000004C5000004C5000004C50000D0
S11300B004C5000004C5000004C5000004C5000018
S11300C048573031424C30313031000031353A3408
S11300D0343A30310000000044656320313220326C
S11300E0303234000000000052502D3737420000F7
S11300F000000000000000000000000000000000FC
S113040027C08FD2A0D34DDC000000000000FFFF06
S1130410BFFFFFFFFFFFFFFFFE88E6BE30A25B8E3B
S113042000B5020093680120DB680340DBB2002BB7
S11304300AD093681B6A9B081840C0B2002803D0F6
S1130440D0690860012000E0002000BDF2B584B04E
S11304500200002001009468E66801239E43012302
S11304600D00EDB21D403543E560049E3678002E44
S113047051D0D169294CA14201D1010012E0D169C6
S1130480274CA14201D219000CE0D169254CA142AC
S113049001D2022106E0D169234CA14201D20321F9
S11304A000E004210C00E4B2042C01D1002033E06C
S11304B06C46617094680194019CE4680C25AC431B
S11304C06D466D78AD000C262E4026430396039CA2
S11304D0019DEC606C4620709068C4681025AC43A4
S11304E06D462D782D011026354025430295029C3A
S11304F0C4601C009568EE680127BE432700FFB264
S11305001F403743EF609068006A84081800204059
S1130510C0B20028F7D0012005B0F0BD00093D00AD
S113052001127A0001366E01015A620200B502001E
S11305309068006A43081800C007C00FC0B20028C2
S113054003D090690860012000E0002000BDF2B5EE
S113055084B005000026A8680124416920000840F1
S1130560C0B200286AD0A868016A20000840C0B25E
S1130570002863D0A8688069010920000840C0B23F
S1130580002802D0012806D00BE069462800FFF7B6
S113059047FF060005E069462800FFF7C7FF06008D
S11305A0FFE73000C0B2002801D1002048E0270056
S11305B0A8684069000A8007800FC0B2002805D0EF
S11305C0022808D004D3032808D00AE0270008E052
S11305D00220070005E00420070002E008200700CD
S11305E0FFE7A868406940084006400EC0B20028F2
S11305F002D18020029000E00290A8684069C00AFD
S11306004007400FC0B2002802D10820019000E04A
S11306100190A8684069810A20000840C0B2401CCB
S113062003900098029948430399484301997943F8
S1130630490002F05AFB0499086026003000C0B259
S113064005B0F0BDFCB502000020040095686E6999
S113065001239E4301232700FFB21F403743019724
S1130660019E6E611E006F463E704E78002E02D0D1
S1130670012E0FD01DE004009568AF691026B74322
S1130680BC462600F6B2360110273E4067463E437C
S1130690AE6111E01C009568AF691026B743BC46F3
S11306A02600F6B2360110273E4067463E43AE614F
S11306B002E004006D462C706C462478002C01D1B5
S11306C0002093E0CC68012C01D104000FE0CC6839
S11306D0022C01D11C000AE0CC68042C01D10224B4
S11306E005E0CC68082C01D1032400E0FF24250098
S11306F0EDB2FF2D01D1002078E06D466C70956855
S11307006E69834F3740BC466E4676783702C02602
S1130710B6003E4067463E436E614F88002F1CD0B2
S11307204D88812D19DA4D88802D01D1050000E016
S11307304D8896680196019E7769FE26B743BC46AC
S11307402E00F6B27700FE263E4067463E43019FE8
S11307507E610F69002F02D11AE0002046E00D6986
S1130760092D15D20D69082D00D0086995686E69A8
S1130770B04F3740BC460600F6B2F702E026B60199
S11307803E4067463E436E618F68012F02D104E00C
S113079000202BE08868022813D18868401E9568E1
S11307A06E69A54F3740BC460600F6B2B6028027F4
S11307B0FF003E4067463E436E610F78002F02D132
S11307C012E0002012E0180095686E690127BE430C
S11307D00700FFB21F4037436F619068056A180035
S11307E02840C0B20028F8D068460078F6BDF3B5BA
S11307F081B0070000242600009478690125C069AF
S1130800010928000840C0B2002818D06946380001
S1130810FFF706FE06003000C0B200280FD078694A
S1130820C069000A4007400F85402900412905D2CC
S1130830009802F05AFA0299086000E0260030009D
S1130840C0B2FEBDFEB5020000206B4618706B46B8
S113085058705369DE691024E443264010256F461E
S11308607F783F012F403743DF618E88012E01D10D
S113087003001EE08B88022B01D1012319E08B8831
S1130880042B01D1022314E08B88082B01D103230C
S11308900FE08B88102B01D104230AE08B88202BD6
S11308A001D1052305E08B88402B01D1062300E00C
S11308B007231E00F6B2072E17D06E4673705669D2
S11308C00196019EF669A54F3740BC466E46767880
S11308D03702E026F6003E4067463E430296029EFB
S11308E0019FFE6101266F463E700E78002E01D0F6
S11308F0012600E006005769F86904403000C0B2E0
S1130900000105402543FD6168460078FEBD0000F6
S1130910FFFCFFFFF3B581B007000024260000941C
S1130920786901258069010928000840C0B20028BF
S113093018D069463800FFF773FD06003000C0B2D6
S113094000280FD078698069000A4007400F85406D
S11309502900412905D2009802F0C7F902990860DC
S113096000E026003000C0B2FEBDFEB5020000204B
S11309706B4618706B46587053699E691024E443A3
S1130980264010256F467F783F012F4037439F61F3
S11309908E88012E01D103001EE08B88022B01D129
S11309A0012319E08B88042B01D1022314E08B88E6
S11309B0082B01D103230FE08B88102B01D10423D2
S11309C00AE08B88202B01D1052305E08B88402B7E
S11309D001D1062300E007231E00F6B2072E17D02C
S11309E06E46737056690196019EB6695B4F374037
S11309F0BC466E4676783702E026F6003E406746EF
S1130A003E430296029E019FBE6101266F463E70E0
S1130A100E78002E01D0012600E006005769B8695F
S1130A2004403000C0B2000105402543BD61684662
S1130A300078FEBDFFC7FFFFFFFBFFFFF3B581B0EA
S1130A400700002426000094786901254069010903
S1130A5028000840C0B2002818D069463800FFF7C3
S1130A6065FD06003000C0B200280FD078694069E7
S1130A70000A4007400F85402900412905D200980B
S1130A8002F033F90299086000E026003000C0B299
S1130A90FEBDFEB5020000206B4618706B46587010
S1130AA053695E691024E443264010256F467F781D
S1130AB03F012F4037435F618E88012E01D103002F
S1130AC01EE08B88022B01D1012319E08B88042BB3
S1130AD001D1022314E08B88082B01D103230FE0FA
S1130AE08B88102B01D104230AE08B88202B01D1A1
S1130AF0052305E08B88402B01D1062300E0072362
S1130B001E00F6B2072E17D06E4673705669019612
S1130B10019E7669114F3740BC466E46767837029F
S1130B20E026F6003E4067463E430296029E019F41
S1130B307E6101266F463E700E78002E01D001269C
S1130B4000E006005769786904403000C0B2000133
S1130B50054025437D6168460078FEBDFFF8FFFF30
S1130B60F3B581B0070000242600009478690125BC
S1130B700069010928000840C0B2002818D069465D
S1130B803800FFF7D3FC06003000C0B200280FD0B5
S1130B9078690069000A4007400F8540290041290F
S1130BA005D2009802F0A1F80299086000E026003E
S1130BB03000C0B2FEBDFEB5020000206B461870C6
S1130BC06B46587053691E691024E443264010256F
S1130BD06F467F783F012F4037431F618E88012E77
S1130BE001D103001EE08B88022B01D1012319E0FF
S1130BF08B88042B01D1022314E08B88082B01D1AC
S1130C0003230FE08B88102B01D104230AE08B8887
S1130C10202B01D1052305E08B88402B01D106232D
S1130C2000E007231E00F6B2072E17D06E4673703D
S1130C3056690196019E3669A14F3740BC466E46FF
S1130C4076783702E026F6003E4067463E43029639
S1130C50029E019F3E6101266F463E700E78002E73
S1130C6001D0012600E006005769386904403000CD
S1130C70C0B20001054025433D6168460078FEBDD1
S1130C80F3B581B00700002426000094786901259B
S1130C90406A010928000840C0B2002818D06946FB
S1130CA03800FFF754FC06003000C0B200280FD013
S1130CB07869406A000A4007400F854029004129AD
S1130CC005D2009802F011F80299086000E02600AD
S1130CD03000C0B2FEBDFEB5020000206B461870A5
S1130CE06B46587053695E6A1024E443264010250D
S1130CF06F467F783F012F4037435F628E88012E15
S1130D0001D103001EE08B88022B01D1012319E0DD
S1130D108B88042B01D1022314E08B88082B01D18A
S1130D2003230FE08B88102B01D104230AE08B8866
S1130D30202B01D1052305E08B88402B01D106230C
S1130D4000E007231E00F6B2072E17D06E4673701C
S1130D5056690196019E766A594F3740BC466E46E5
S1130D6076783702E026F6003E4067463E43029618
S1130D70029E019F7E6201266F463E700E78002E11
S1130D8001D0012600E006005769786A044030006B
S1130D90C0B20001054025437D6268460078FEBD6F
S1130DA0F3B581B00700002426000094786901257A
S1130DB0006A010928000840C0B2002818D069461A
S1130DC03800FFF7C4FB06003000C0B200280FD083
S1130DD07869006A000A4007400F854029004129CC
S1130DE005D2009801F081FF0299086000E0260016
S1130DF03000C0B2FEBDFEB5020000206B46187084
S1130E006B46587053691E6A1024E443264010252B
S1130E106F467F783F012F4037431F628E88012E33
S1130E2001D103001EE08B88022B01D1012319E0BC
S1130E308B88042B01D1022314E08B88082B01D169
S1130E4003230FE08B88102B01D104230AE08B8845
S1130E50202B01D1052305E08B88402B01D10623EB
S1130E6000E007231E00F6B2072E17D06E467370FB
S1130E7056690196019E366A114F3740BC466E464C
S1130E8076783702E026F6003E4067463E430296F7
S1130E90029E019F3E6201266F463E700E78002E30
S1130EA001D0012600E006005769386A044030008A
S1130EB0C0B20001054025433D6268460078FEBD8E
S1130EC0FFF8FFFF70B504000E000025606900689C
S1130ED0000E8007800FC0B2002805D002280FD072
S1130EE008D3032812D017E031002000FFF71EFBBF
S1130EF0050011E031002000FFF792FA05000BE035
S1130F0031002000FFF723FB050005E0310020003D
S1130F10FFF70CFB0500FFE72800C0B270BDF0B579
S1130F2002004878012801D100230AE0487800280B
S1130F3001D1012305E04878022801D1022300E011
S1130F40FF231800C0B2FF2801D1002017E01C00C5
S1130F5050690668934D35402600F6B23704C02622
S1130F60B6023E402E43066050690068000E8007BA
S1130F70800F1C00C0B2E4B2A042F5D10120F0BD44
S1130F80F8B504000E00002569462000FFF79AFF1B
S1130F9007003800C0B2002801D100200BE0E0684F
S1130FA000680107090F0098C9B2491C01F09DFEB1
S1130FB030603800C0B2F2BD30B502008888002825
S1130FC010D0888811280DDA8C88641ED3681868BC
S1130FD00F25A8432500EDB22D072D0F05431D60F5
S1130FE0012000E0002030BDF8B504000E0000250B
S1130FF069462000FFF7C4FF07003800C0B200288C
S113100001D100200CE060690068000A0107090FA3
S11310100098C9B2491C01F068FE30603800C0B2C3
S1131020F2BD70B502008888002812D08888112883
S11310300FDA8C88641E53691D685B4828402500BC
S1131040EDB22E02F0252D01354005431D6001202F
S113105000E0002070BDF8B504000F0000252E004C
S11310602069C8214058000C8007800FC0B20028B6
S113107005D002280FD008D3032812D017E0694600
S11310802000FFF753FA060011E069462000FFF73D
S1131090C7F906000BE069462000FFF758FA06007E
S11310A005E069462000FFF741FA0600FFE730003B
S11310B0C0B2002801D1002019E02069C82140589D
S11310C001090800C007C00FC0B200280CD0206975
S11310D0C8214058000A0107090F0098C9B2491CE9
S11310E001F003FE386000E02E003000C0B2F2BD13
S11310F0FCB502004878012801D100230AE04878B1
S1131100002801D1012305E04878022801D10223F7
S113111000E0FF231800C0B2FF2801D100203FE007
S1131120888800283BD08888112838DA68460370FC
S11311301069C82405591B4C2C406D462D782D048C
S1131140C026B6022E4026430196019CC825445170
S11311508C88641E1569C826AE59134F3740BC46A7
S11311602600F6B23702F02636013E4067463E437B
S1131170C827EE510F78002F01D0012400E000248D
S11311801569C82028581026B0432600F6B2360147
S113119010273E400643C8202E50012000E00020C6
S11311A0F6BD0000FFFFFCFFFFF0FFFFF8B50400F1
S11311B00F006069406801090800C007C00FC0B291
S11311C0002801D100209BE0002005000090606908
S11311D007264068000C3040C0B2002843D1606943
S11311E04068C00C3040C0B200280BD0022815D093
S11311F00ED304281ED017D3062827D020D30728BF
S11312002AD02FE069462000FFF725FF050066E09D
S113121069462000FFF704F9050060E069462000F4
S1131220FFF784F905005AE069462000FFF78FF9BB
S1131230050054E069462000FFF7A2FE05004EE0D9
S113124069462000FFF7D0FE050048E0694620000B
S1131250FFF7CDFA050042E069462000FFF7EEFBF8
S113126005003CE03BE060694068000C3040C0B2DF
S113127001280AD033D3032813D00CD305281CD05B
S113128015D3072825D01ED329E069462000FFF78F
S1131290F7FC050023E06946200000F038FA050059
S11312A01DE06946200000F00BFA050017E06946CE
S11312B0200000F0DEF9050011E06946200000F08E
S11312C067FD05000BE069462000FFF72FF90500D4
S11312D005E069462000FFF729F90500FFE728002B
S11312E0C0B201280AD160694068000A0640310092
S11312F00098C9B2491C01F0F8FC38602800C0B25B
S1131300F2BDF2B582B0010001206A4610700020DF
S113131002004B695C681025AC431500EDB22D0149
S11313201026354025435D60029C6478002C40D033
S1131330012C5DD0022C7AD0032C00D1D4E0052CF2
S113134000D1F0E0072C00D10CE10A2C00D18DE093
S11313500B2C00D1A9E00C2C0CD00F2C00D12BE1CC
S1131360102C00D11AE1112C00D109E11A2C00D162
S113137030E13DE102004B695D68B94C2C40150039
S1131380EDB22D04E026F6022E4026430196019C80
S11313905C6004004D696E68B24F3740BC4626005D
S11313A0F6B2F704E026B6033E4067463E436E605D
S11313B021E102004B695D68A94C2C401500EDB297
S11313C02D04E026F6022E4026430196019C5C6023
S11313D001244D696E68A34F3740BC462600F6B21F
S11313E0F704E026B6033E4067463E436E6002E1E2
S11313F002004B695D689A4C2C401500EDB22D0437
S1131400E026F6022E4026430196019C5C600224ED
S11314104D696E68934F3740BC462600F6B2F70418
S1131420E026B6033E4067463E436E60E3E00200BA
S11314304B695D688A4C2C401500EDB22D04E02602
S1131440F6022E4026430196019C5C6003244D69FC
S11314506E68844F3740BC462600F6B2F704E02697
S1131460B6033E4067463E436E60C4E002004B69EB
S11314705D687B4C2C401500EDB22D04E026F6028D
S11314802E4026430196019C5C6004244D696E68DD
S1131490744F3740BC462600F6B2F704E026B60384
S11314A03E4067463E436E60A5E002004B695D68BE
S11314B06B4C2C401500EDB22D04E026F6022E40B4
S11314C026430196019C5C6005244D696E68654F56
S11314D03740BC462600F6B2F704E026B6033E4089
S11314E067463E436E6086E002004B695D685C4C73
S11314F02C401500EDB22D04E026F6022E402643C2
S11315000196019C5C6006244D696E68554F374016
S1131510BC462600F6B2F704E026B6033E40674612
S11315203E436E6067E002004B695D684C4C2C40A2
S11315301500EDB22D04E026F6022E402643019656
S1131540019C5C6007244D696E68464F3740BC4679
S11315502600F6B2F704E026B6033E4067463E4353
S11315606E6048E001224B695D683D4C2C401500DB
S1131570EDB22E04E025ED02354025435D603AE0EE
S113158002224B695D68364C2C401500EDB22E04E6
S1131590E025ED02354025435D602CE003224B69D4
S11315A05D682F4C2C401500EDB22E04E025ED02B1
S11315B0354025435D601EE004224B695D68284C7C
S11315C02C401500EDB22E04E025ED0235402543F4
S11315D05D6010E005224B695D68214C2C401500CC
S11315E0EDB22E04E025ED02354025435D6002E0B6
S11315F002006B461A706A461278002A1AD0029AC0
S11316009288002A13D0029A9288092A0FDA029A41
S11316109288521E4B695D687F4C2C401500EDB2D8
S11316202E02E025ED00354025435D6002E0020016
S11316306B461A70029A1278002A01D0012200E047
S113164002004B6958681024A0431400E4B224013A
S113165010252C4004435C6068460078FEBD000001
S1131660FFFFF8FFFFFFC7FF0200106A08600120B8
S1131670704700B502005068806C03091800C00769
S1131680C00FC0B2002804D0FA20800008600120F6
S113169000E0002000BD70B502000878002801D0E9
S11316A0012400E000245368986C1025A843250009
S11316B0EDB22D011026354005439D64012070BD17
S11316C000B502005068406C03091800C007C00F41
S11316D0C0B2002804D0FA20C0010860012000E054
S11316E0002000BD70B502000878002801D0012454
S11316F000E000245368586C1025A8432500EDB27F
S11317002D011026354005435D64012070BD0200A3
S1131710FA20400208600120704770B504000E00F2
S1131720002561680120496809090140C9B20029FE
S113173001D100201AE061684968090C0140C9B26E
S1131740002905D131002000FFF71AFC05000BE049
S113175061684968090C0840C0B2012804D131000D
S1131760200000F02FF905002800C0B270BDF2B5CA
S113177082B0010000206A46107005004C6866685B
S11317801022D243164010232F00FFB23F011F4006
S113179037436760029E76780A2E11D16C466070DA
S11317A04C6866681D4D35406E4676783604802751
S11317B07F023E402E43666001256F463D7018E06F
S11317C0029C6478182C14D1012425004E680196DB
S11317D0019E7668114F3740BC462E00F6B236049F
S11317E080277F023E4067463E43019F7E606F46EE
S11317F03C70029C2478002C01D0012400E00400F9
S11318004D68686802402000C0B2000103401343E1
S11318106B6068460078FEBDFFF8FFFFFFFFFEFF28
S113182070B504000E000025606880680109080096
S1131830C007C00FC0B2002804D031002000FFF759
S1131840D3FB05002800C0B270BD70B50200087853
S1131850002801D0012400E0002453689868102572
S1131860A8432500EDB22D011026354005439D60A7
S1131870012070BD70B504000E0000256068C068CA
S113188001090800C007C00FC0B2002804D031000D
S11318902000FFF7A9FB05002800C0B270BD70B599
S11318A002000878002801D0012400E000245368D5
S11318B0D8681025A8432500EDB22D011026354027
S11318C00543DD60012070BD70B504000E000025E5
S11318D06068006901090800C007C00FC0B2002891
S11318E004D031002000FFF77FFB05002800C0B2C0
S11318F070BD70B502000878002801D0012400E012
S11319000024536818691025A8432500EDB22D0161
S11319101026354005431D61012070BD70B50400DB
S11319200E0000256068406901090800C007C00F67
S1131930C0B2002804D031002000FFF755FB050099
S11319402800C0B270BD70B502000878002801D02C
S1131950012400E00024536858691025A843250099
S1131960EDB22D011026354005435D61012070BDA7
S113197070B504000E000025606880690109080044
S1131980C007C00FC0B2002804D031002000FFF708
S11319902BFB05002800C0B270BD70B502000878AA
S11319A0002801D0012400E0002453689869102520
S11319B0A8432500EDB22D011026354005439D6155
S11319C0012070BDF8B505000F0000200400009050
S11319D06868C06901090800C007C00FC0B20028C8
S11319E001D1002054E068680726C069000C30402B
S11319F0C0B200280BD0022815D00ED304281ED064
S1131A0017D3062827D020D307282AD02FE06946E9
S1131A102800FFF713F8040029E069462800FEF7C0
S1131A20E6FE040023E069462800FFF729F90400D4
S1131A301DE069462800FFF76AFE040017E06946C6
S1131A402800FFF716FE040011E069462800FFF79E
S1131A5037FE04000BE069462800FFF705FE04008A
S1131A6005E069462800FEF7E9FF0400FFE72000CF
S1131A70C0B200280AD06868C069000A0640310074
S1131A80C9B2491C009801F030F938602000C0B296
S1131A90F2BDF3B50100012002006B461A7000226A
S1131AA014004D68EE6910239E4310232700FFB2F3
S1131AB03F011F403743EF61019E7678032E1CD00F
S1131AC0052E0AD0072E28D00E2E66D00F2E44D015
S1131AD0102E52D0112E30D06FE014004D68EE69F4
S1131AE0AA4F3740BC462600F6B23704E026F60279
S1131AF03E4067463E43EE6162E004004D68EE6995
S1131B00A24F3740BC462600F6B23704E026F60260
S1131B103E4067463E43EE6152E002244D68EE6962
S1131B209A4F3740BC462600F6B23704E026F60248
S1131B303E4067463E43EE6142E003244D68EE6951
S1131B40924F3740BC462600F6B23704E026F60230
S1131B503E4067463E43EE6132E004244D68EE6940
S1131B608A4F3740BC462600F6B23704E026F60218
S1131B703E4067463E43EE6122E005244D68EE692F
S1131B80824F3740BC462600F6B23704E026F60200
S1131B903E4067463E43EE6112E006244D68EE691E
S1131BA07A4F3740BC462600F6B23704E026F602E8
S1131BB03E4067463E43EE6102E014006D462C70E1
S1131BC0019CA488002C15D0019CA488092C11DA4E
S1131BD0019CA488641E4D68EE69C04F3740BC4622
S1131BE02600F6B23702E026F6003E4067463E4342
S1131BF0EE6102E014006D462C70019C2478002CE8
S1131C0001D00200FFE74C68E0691025A8431500E5
S1131C10EDB22D012B400343E36168460078F6BD25
S1131C2070B504000E00002561680120096A0909E5
S1131C300140C9B2002901D1002026E06168096A87
S1131C40090C8907890FC9B2002905D002290FD0D0
S1131C5008D3032912D016E031002000FEF7EEFE6F
S1131C60050010E031002000FFF70AF805000AE043
S1131C7031002000FEF7BBFD050004E0FA21490213
S1131C8031600500FFE72800C0B270BDF2B582B034
S1131C900100012002006B461A7000226B465A7044
S1131CA04D682E6A1023DB431E4010246F467F7854
S1131CB03F01274037432F62029E7678032E2AD0B5
S1131CC0052E04D0072E13D0112E37D049E06D46CF
S1131CD06A704D682E6AC94F3740BC466E467678A6
S1131CE03704C026B6023E4067463E432E623AE0C1
S1131CF005004E680196019E366AC04F3740BC46C7
S1131D002E00F6B23704C026B6023E4067463E4374
S1131D10019F3E6227E002254E680196019E366AC5
S1131D20B64F3740BC462E00F6B23704C026B60282
S1131D303E4067463E43019F3E6214E003254E68E1
S1131D400196019E366AAD4F3740BC462E00F6B26E
S1131D503704C026B6023E4067463E43019F3E62BA
S1131D6001E06D462A70029D2D78002D01D00200FD
S1131D70FFE74D68286A03401000C0B20001044028
S1131D801C432C6268460078FEBD0000FFFFF8FF8C
S1131D9070B504000E0000256068806A010908001F
S1131DA0C007C00FC0B2002801D1002027E060683E
S1131DB0806A000C8007800FC0B2002805D002287A
S1131DC00FD008D3032812D017E031002000FFF70A
S1131DD077FC050011E031002000FFF745FC050009
S1131DE00BE031002000FFF744FC050005E0310062
S1131DF02000FFF73EFC0500FFE72800C0B270BDDD
S1131E00F2B582B0010000206A46107005004C68EB
S1131E10A66A1022D243164010232F00FFB23F01BE
S1131E201F403743A762029E7678102E11D16C466C
S1131E3060704C68A66A714D35406E4676783704FA
S1131E40C026B6023E402E43A66201256F463D7071
S1131E5031E0029C64780E2C15D1012425004E68D3
S1131E600196019EB66A654F3740BC462E00F6B215
S1131E703704C026B6023E4067463E43019FBE6219
S1131E806F463C7017E0029C64780F2C13D1022437
S1131E904D68AE6A594F3740BC462600F6B2370447
S1131EA0C026B6023E4067463E430196019EAE629E
S1131EB001266F463E70029C2478002C01D0012438
S1131EC000E004004D68A86A02402000C0B200018E
S1131ED003401343AB6268460078FEBDFFF8FFFF82
S1131EE070B504000E00002561680120096B090C1F
S1131EF00140C9B2002905D131002000FFF774F870
S1131F0005000BE06168096B090C0840C0B20128A8
S1131F1004D131002000FFF7FAFB05002800C0B20D
S1131F2070BDF0B50200002318004C780B2C0CD1C6
S1131F305468266B9D4D35401E00F6B2370480264A
S1131F40760237402F4327630FE04B78112B0CD1D7
S1131F5001235468266B954D35401E00F6B23704B4
S1131F608026760237402F432763C0B2F0BD70B598
S1131F7004000E00002561680120496B090C014032
S1131F80C9B2002905D131002000FFF72DF8050062
S1131F900BE06168496B090C0840C0B2012804D108
S1131FA031002000FFF7B3FB05002800C0B270BD6C
S1131FB0F0B50200002318004C780B2C0CD15468A7
S1131FC0666B7A4D35401E00F6B2370480267602E1
S1131FD037402F4367630FE04B78112B0CD101235B
S1131FE05468666B714D35401E00F6B23704802686
S1131FF0760237402F436763C0B2F0BDFFFFFCFF9A
S113200070B504000E00002561680120896B090C7D
S11320100140C9B2002905D131002000FEF7E4FFD8
S113202005000BE06168896B090C0840C0B2012807
S113203004D131002000FFF76AFB05002800C0B27C
S113204070BDF0B50200002318004C780B2C0CD1A5
S11320505468A66B554D35401E00F6B237048026F1
S1132060760237402F43A7630FE04B78112B0CD136
S113207001235468A66B4D4D35401E00F6B237045B
S11320808026760237402F43A763C0B2F0BD70B5F7
S113209004000E00002561680120C96B090C014091
S11320A0C9B2002905D131002000FEF79DFF0500CB
S11320B00BE06168C96B090C0840C0B2012804D167
S11320C031002000FFF723FB05002800C0B270BDDB
S11320D0F0B50200002318004C780B2C0CD1546886
S11320E0E66B324D35401E00F6B237048026760288
S11320F037402F43E7630FE04B78112B0CD10123BA
S11321005468E66B294D35401E00F6B2370480262C
S1132110760237402F43E763C0B2F0BD70B50400C8
S11321200E00002561680120096C090C0140C9B248
S1132130002905D131002000FEF756FF05000BE011
S11321406168096C090C0840C0B2012804D131004F
S11321502000FFF7DCFA05002800C0B270BDF0B51E
S11321600200002318004C780B2C0CD15468266C08
S11321700E4D35401E00F6B23704802676023740F5
S11321802F4327640FE04B78112B0CD101235468A3
S1132190266C064D35401E00F6B2370480267602C2
S11321A037402F432764C0B2F0BD0000FFFFFEFF9D
S11321B070B504000E00002521680120C9680909D2
S11321C00140C9B2002905D131002000FEF70CFFFF
S11321D005000AE02168C96809090140C9B201295A
S11321E003D1FA214902316005002800C0B270BD54
S11321F0F0B50200002318004C780B2C0DD11468A4
S1132200E5681026B5431E00F6B2360110273E409D
S11322102E43E6600125280012E04B78112B0FD1E4
S113222001231C001568EF681026B743BC4626003E
S1132230F6B2360110273E4067463E43EE60180072
S1132240C0B2F0BD38B505000C002869006801096A
S11322500800C007C00FC0B2002801D1002003E06D
S113226021002800FEF78CFE32BD70B5020008780C
S1132270002801D0012400E0002413691868102507
S1132280A8432500EDB22D011026354005431D60FD
S1132290012070BD38B505000C00286940680109AB
S11322A00800C007C00FC0B2002801D1002003E01D
S11322B021002800FEF798FE32BD70B502000878B0
S11322C0002801D0012400E0002413695868102577
S11322D0A8432500EDB22D011026354005435D606D
S11322E0012070BD38B505000C002869006901099A
S11322F00800C007C00FC0B2002801D1002003E0CD
S113230021002800FEF770FE32BD70B50200087887
S1132310002801D0012400E0002413691869102565
S1132320A8432500EDB22D011026354005431D615B
S1132330012070BD38B505000C0028694069010909
S11323400800C007C00FC0B2002801D1002003E07C
S113235021002800FEF748FE32BD70B5020008785F
S1132360002801D0012400E00024136958691025D5
S1132370A8432500EDB22D011026354005435D61CB
S1132380012070BD38B505000C0028698069010979
S11323900800C007C00FC0B2002801D1002003E02C
S11323A021002800FEF7ECFD32BD70B5020008786C
S11323B0002801D0012400E0002413699869102545
S11323C0A8432500EDB22D011026354005439D613B
S11323D0012070BD38B505000C002869C0690109E9
S11323E00800C007C00FC0B2002801D1002003E0DC
S11323F021002800FEF7F8FD32BD70B50200087810
S1132400002801D0012400E000241369D8691025B4
S1132410A8432500EDB22D01102635400543DD61AA
S1132420012070BDF2B582B0060030690124006A53
S1132430010920000840C0B2002801D1002037E083
S11324402000694608710027009730690325006A57
S1132450000C2840C0B2002805D002280FD008D3B1
S1132460032812D017E069463000FEF75FF8070032
S113247011E069463000FDF7D3FF07000BE0694621
S11324803000FEF764F8070005E069463000FEF707
S11324904DF80700FFE73069006A000A0540AC40C8
S11324A00098210000F021FC029908603800C0B2B5
S11324B0FEBDFEB5020000206B4618706B465870D6
S11324C013691E6A1024E443264010256F467F7862
S11324D03F012F4037431F624E78012E01D1030084
S11324E00AE04B78002B01D1012305E04B78022B45
S11324F001D1022300E0FF231E00F6B2FF2E17D005
S11325006E46737016690196019E366A844F374091
S1132510BC466E4676783704C026B6023E4067460F
S11325203E430296029E019F3E6201266F463E7024
S11325306E463678002E36D08E88012E01D10600E4
S11325400FE08E88022E01D101260AE08E88042E27
S113255001D1022605E08E88082E01D1032600E071
S1132560FF266F467E706E467678FF2E19D06E4633
S113257076786F46BE7016690296029E376A694E77
S11325803E400196019FBC466E46B6783702C0268F
S1132590B6003E4067463E430196019E029F3E625E
S11325A001E06E4630700E78002E01D0012600E066
S11325B006001769386A04403000C0B200010540C3
S11325C025433D6268460078FEBD38B505000C0021
S11325D02869806A01090800C007C00FC0B200283A
S11325E001D1002003E021002800FEF7FDFC32BDEC
S11325F070B502000878002801D0012400E000240E
S11326001369986A1025A8432500EDB22D01102600
S1132610354005439D62012070BD70B505000C0076
S113262028690126006B00093040C0B2002801D19E
S1132630002023E02869006B000C8007800FC0B2E3
S1132640002805D002280DD007D303280FD013E0AB
S113265021002800FEF7F2F90FE021002800FEF720
S1132660C6F80AE021002800FEF70AFB05E0210075
S11326702800FEF7E3F900E00020C0B270BDFEB50B
S1132680020000206B4618706B46587013691E6B6D
S11326901024E443264010256F467F783F012F40E5
S11326A037431F634E78052E01D103000AE04B78AF
S11326B0032B01D1012305E04B78072B01D1022321
S11326C000E0FF231E00F6B2FF2E17D06E46737093
S11326D016690196019E366B114F3740BC466E4613
S11326E076783704C026B6023E4067463E430296DB
S11326F0029E019F3E6301266F463E700E78002EB7
S113270001D0012600E006001769386B0440300050
S1132710C0B20001054025433D6368460078FEBD14
S1132720FFFFFCFFFFFCFFFF0200506A086001206E
S113273070470200906A0860012070470200D06A66
S113274008600120704770B505000C000126286957
S1132750A0214058000C4007400FC0B200280BD005
S1132760022813D00DD304281AD014D3062821D05C
S11327701BD307281ED022E021002800FFF7D4FF36
S11327801EE021002800FFF7D4FF19E021002800F3
S1132790FFF7D4FF14E021002800FEF7E1F90FE071
S11327A021002800FEF7B6F80AE021002800FEF711
S11327B0F7FA05E021002800FEF7D2F900E0002036
S11327C0C0B270BDF0B50200012318004C78042C8F
S11327D049D0062C37D0082C55D02A2C04D02B2CC9
S11327E012D02C2C1FD05EE000231469A02566595A
S11327F0AD4D35401E00F6B23704E026F6023E40E9
S11328002E43A025665150E01469A0256659A64DB3
S113281035401E00F6B23704E026F6023E402E4351
S1132820A025665141E002231469A02566599E4DF6
S113283035401E00F6B23704E026F6023E402E4331
S1132840A025665131E003231469A0256659964DED
S113285035401E00F6B23704E026F6023E402E4311
S1132860A025665121E004231469A02566598E4DE4
S113287035401E00F6B23704E026F6023E402E43F1
S1132880A025665111E005231469A0256659864DDB
S113289035401E00F6B23704E026F6023E402E43D1
S11328A0A025665101E000231800C0B2F0BD70B548
S11328B005000C0001262869A4214058000C40079B
S11328C0400FC0B200280BD0022813D00DD3042827
S11328D01AD014D3062821D01BD307281ED022E0F7
S11328E021002800FFF720FF1EE021002800FFF749
S11328F020FF19E021002800FFF720FF14E0210049
S11329002800FEF72DF90FE021002800FEF702F859
S11329100AE021002800FEF743FA05E02100280020
S1132920FEF71EF900E00020C0B270BDF0B5020051
S1132930012318004C78042C49D0062C37D0082CDD
S113294055D02A2C04D02B2C12D02C2C1FD05EE076
S113295000231469A4256659534D35401E00F6B270
S11329603704E026F6023E402E43A425665150E08B
S11329701469A42566594C4D35401E00F6B237043F
S1132980E026F6023E402E43A425665141E0022390
S11329901469A4256659444D35401E00F6B2370427
S11329A0E026F6023E402E43A425665131E003237F
S11329B01469A42566593C4D35401E00F6B237040F
S11329C0E026F6023E402E43A425665121E004236E
S11329D01469A4256659344D35401E00F6B23704F7
S11329E0E026F6023E402E43A425665111E005235D
S11329F01469A42566592C4D35401E00F6B23704DF
S1132A00E026F6023E402E43A425665101E0002351
S1132A101800C0B2F0BD70B505000C00012006001E
S1132A202969C0228958090C0840C0B2002802D084
S1132A30012805D009E021002800FEF741FE05E049
S1132A4021002800FEF710FE00E00020C0B270BD97
S1132A50F0B50200012318004C780E2C11D0102C74
S1132A601ED100231469C02566598E4D35401E00C1
S1132A70F6B2360480277F023E402E43C0256651BD
S1132A8010E01469C0256659864D35401E00F6B223
S1132A90360480277F023E402E43C025665101E064
S1132AA000231800C0B2F0BDFFFFF8FF70B50500A9
S1132AB00C00012006002969C4228958090C084029
S1132AC0C0B2002802D0012805D009E02100280066
S1132AD0FEF7F6FD05E021002800FEF7C5FD00E045
S1132AE00020C0B270BDF0B50200012318004C787C
S1132AF00E2C11D0102C1ED100231469C425665944
S1132B00684D35401E00F6B2360480277F023E40F1
S1132B102E43C425665110E01469C4256659614DDD
S1132B2035401E00F6B2360480277F023E402E4315
S1132B30C425665101E000231800C0B2F0BD38B5C9
S1132B4005000C002869CC21405801090800C00781
S1132B50C00FC0B2002801D1002003E021002800EA
S1132B60FEF70EFA32BD70B502000878002801D0D5
S1132B70012300E000231469CC2020581025A84329
S1132B801D00EDB22D01102635400543CC20255003
S1132B90012070BDFEB50899099A0A9B0B9C009D03
S1132BA00560019D4560029D8560C16002614361CD
S1132BB0256885616568C561A568056200252E00E4
S1132BC02E00F6B2032E0BD22E00F6B2B600A619D2
S1132BD0F6682F00FFB2BF00C7197E626D1CEFE7D5
S1132BE0F7BDF8B506000C0017002000C0B232286B
S1132BF001DB002011E000252B4A2000C0B2C000F8
S1132C001058002807D0390030002300DBB2DB0065
S1132C10D258904705002800C0B2F2BDF4B588B080
S1132C2004000F003800C0B2322801DB002037E076
S1132C3000252E001C4A3800C0B2C000101840689D
S1132C4000282BD0194807906068069007980699C9
S1132C508023C85016480590A068049005980499EC
S1132C600866144803902068029003980299802310
S1132C70C850089920003B00DBB2DB00D218526830
S1132C809047060001956068019980228150009563
S1132C90A168009A0A6622688023D5503000C0B229
S1132CA009B0F0BDFFFFFEFF3CB80000524553558C
S1132CB0202096194B4D4352F446002804D449422F
S1132CC000F013F8404260474042002905D45FD029
S1132CD000F00BF8404249426047494200F005F8D1
S1132CE04942604703460B43E6D40022030A8B4261
S1132CF00BD203098B4219D243088B422ED2411ABC
S1132D0000D20146524110467047FF2209023FD0CB
S1132D1012068B4205D3121209028B4201D31212FE
S1132D20090203098B4219D300E0090AC3098B4243
S1132D3001D3CB01C01A524183098B4201D38B01C9
S1132D40C01A524143098B4201D34B01C01A52416C
S1132D5003098B4201D30B01C01A5241C3088B42B1
S1132D6001D3CB00C01A524183088B4201D38B009C
S1132D70C01A524143088B4201D34B00C01A52413E
S1132D80884200D3401A5241CFD2014610467047C0
S1132D9008B500F001F808BD7047FEE700B5010072
S1132DA000200A00D2B2002A05D0022A09D005D395
S1132DB0032A09D00AE01022100007E018221000AC
S1132DC004E02822100001E048221000C0B200BD37
S1132DD0F8B505000C002868060080360027684610
S1132DE007703800C0B2FFF7D9FF0100C9B28908E3
S1132DF00800C0B2220092B2504380003018F2BDE5
S1132E0000B5010000200A00D2B2002A082A0ED917
S1132E10093A0ED0521E0FD0521E10D0521E11D09D
S1132E20521E12D0521E13D0521E14D016E00800A7
S1132E3014E00C22100011E0102210000EE0142205
S1132E4010000BE01822100008E02022100005E01A
S1132E503022100002E040221000FFE7C0B200BDA3
S1132E60F8B505000C0000206946487069460870F2
S1132E70210089B22800FFF7ABFF06003068000C80
S1132E8007073F0F3800C0B2FFF7BAFFC0B2F2BD68
S1132E9070B500231400E4B2002C0CD00468C025E3
S1132EA0ED03254305604468640F6407CD00ED0815
S1132EB0254345600BE00468BC4D2540056044682B
S1132EC0BB4E26408C04BB4D25403543456070BD48
S1132ED010B40268B84B1340036002680B00DBB205
S1132EE01B04F02424031C401443046010BC7047EA
S1132EF000B502685200520802600268AF4B1340EA
S1132F0003600A00D2B2002A09D0026880231B069B
S1132F101343036002688023DB051343036000BD91
S1132F2000B50A00D2B2002A06D10268A44B1340AD
S1132F300360026802600CE00A00D2B2012A08D1E0
S1132F4002689F4B1340036002688023DB04134331
S1132F50036000BD30B50268803200231D001C00F0
S1132F60057EED01AC4205D2A500551929000B6080
S1132F70641CF5E730BDF8B4924982688023D150CF
S1132F8001234468256D2026B5431E00F6B2760160
S1132F9020273E402E430096009D25650025866827
S1132FA08027F551F1BC7047F8B4864982688023C4
S1132FB0D15001234468256D1026B5431E00F6B296
S1132FC0360110273E402E430096009D25650025BE
S1132FD086688027F551F1BC7047F2B40599069CC8
S1132FE0079D089E37780776009F076042608360DC
S1132FF0C16004614561F1BC704730B50022110025
S11330008260026142618261C260C2614262826224
S1133010C2620262012303701300C37013000371C0
S11330200023DB4343638363C363036414004425C5
S113303044551400452544551400C8254455082416
S11330404625445514002100C9B2202906DA21007E
S1133050C9B2890041188B64641CF4E71100417003
S11330601100817011003023C1541100C923C154CF
S11330701100CA23C1541100CB23C1541100D5231C
S1133080C1541100D423C1541100D623C1541100DA
S1133090D723C1541100CC23C154D021425030BD98
S11330A0F0B50024210002681368444D1D400B0054
S11330B0DBB29B078026F60533402B43136005687B
S11330C02E68414F3740BC462600F6B236078027AB
S11330D07F053E4067463E432E60016809680A0E3C
S11330E01100C907C90FC9B20029F6D1F0BDF8B55E
S11330F00400206801250068000D2840C0B20028A3
S113310014D0002021680A68520052080300DBB280
S1133110DB0713430B6020680068000D2840C0B231
S1133120002803D02000FFF73FFFF4E728002168C0
S11331300B68264A1A400300DBB25B068026B604FD
S1133140334013430B6020680068400E2840C0B22F
S11331500028F8D16846057020680168174A0A40BB
S11331606946097889078023DB051940114301600A
S11331702A0023681E68144F3740BC461600F6B276
S1133180360780277F053E4067463E431E60206821
S11331900068000E2840C0B20028F8D020680068FB
S11331A0C00E2840C0B20028F1D0F1BDFFFF9FFF40
S11331B0FFFF03E00000FC1FFFFFF0FFFFFFFFBF66
S11331C0FFFFFFF052455355FFFFFFEFFFFFFFFDE9
S11331D0F8B594B007000C0016003100C9B289B2EA
S11331E03800FFF7F5FD0500227A61682800FFF733
S11331F04FFEA17A2800FFF76BFEE17A2800FFF763
S113320077FE617A2800FFF78BFE207B002805D02B
S11332106846067101A9380000F009FD607A0128AA
S11332200AD1206969460E7039686A46127892009C
S11332308A1888231B01D05015B0F0BDF0B58DB0AD
S113324005000E0000206946487000206946087099
S11332502800FFF790FE012029680A6852005208EE
S11332600300DBB2DB0713430B6028680068010D21
S11332700800C007C00FC0B20028F6D030786946F5
S113328048712868029002984068CE490140684617
S1133290407940038022920110400843059005982C
S11332A0029948602800FFF722FF0120694608714F
S11332B02F683968C448084069460979C9058022DD
S11332C012041140014304910498386001206946B6
S11332D0C8702C68616BBD4808406946C978090705
S11332E08022520511400143039103986063280032
S11332F0FFF730FE3020305CFFF750FD69468870E0
S113330068468078002809D0802080006946897842
S1133310FFF7EBFC297E48436946487068464078CD
S11333206946087128680690069800687F218843DA
S1133330694609794906490E01430C910C9806998E
S1133340086001206946C870286805900598006DDA
S1133350400040086946C978C90701430B910B989E
S113336005990865CE48B16809186A46D18129686B
S1133370049104990A6DCB4911406A46D2895205D9
S1133380C94B13400B430A930A99049A1165F168D7
S113339009186A46918129680B6DC44A1A406B4624
S11333A09B891B04F82464031C4014430994099A60
S11333B00A65326912186B465A812A68146DBC4B2F
S11333C023406C466489A702FC2424023C401C432D
S11333D00894089B136573691B186C4623812B683A
S11333E01C6DB44F2740BC466C4624896701F82401
S11333F0A4003C4067463C430794079C1C65B469A1
S113340020186C46E0802868046D1F27BC436F4673
S1133410FF88FF06FF0E27430765F478002C6ED063
S113342001206946887128680268A34911406A46E8
S11334309279520780239B051A400A430692069903
S1133440016031796A46517129680B68CB4A1A4088
S11334506B465B79DB0380242402234013430593EA
S1133460059A0A60326C04922A680392049A039BB8
S11334709A644422B25C6B461A712A681468C04B81
S113348023406C4624792702C024A4003C401C43FA
S11334900294029B13604523F35C6C46E3702B6833
S11334A05C6BB84F2740BC466C46E4782706F02492
S11334B024053C4067463C435C63C827F75D012F05
S11334C03BD1002069460870684600784621715C4B
S11334D0884232D26846007880003018806C694691
S11334E009782A680B00DBB29B00D31888242401D6
S11334F018516B461B785B1C6C462370E4E7002074
S113350029680B686C4A1A400300DBB25B0780240D
S1133510A405234013430193019A0A6000222B68F7
S11335201C68964F2740BC461400E4B2E40380278D
S11335303F023C4067463C431C60706B0390286824
S113354003990161B16B02912968029A4A61F26B95
S113355001922A68019B9361C823F35C6C46E37073
S11335602B681C68BC4F2740BC466C46E478240496
S113357080277F023C4067463C431C60C927F75DB7
S1133580002F25D0002029680B68B44A1A40030094
S1133590DBB25B048024A402234013430193019A09
S11335A00A6001222B685C68AD4F2740BC461400BA
S11335B0E4B2240380277F013C4067463C435C60BF
S11335C024E000BFFFDFFFFFFFFF7FFFFFFFFFEFF0
S11335D0012029680B68A14A1A400300DBB25B048E
S11335E08024A402234013430193019A0A60002219
S11335F02B685C689A4F2740BC461400E4B224034D
S113360080277F013C4067463C435C60D420305CAB
S1133610002853D0012001006A46917129680B6883
S1133620904A1A406B469B799B058024E40323400F
S113363013430593059A0A6002006B465A712A687F
S11336401468894B23406C466479A4068027FF04E0
S11336503C401C430494049B136003006C46237198
S11336602B681C68814F2740BC466C462479A4040F
S11336708027FF023C4067463C430394039C1C6044
S113368004006F46FC706C690294029CA46C0127D0
S1133690BC436F46FF7838402043029CA06453E04B
S11336A0FFFF0000FFFF1F800000E07FFFFFE0FF3F
S11336B0FF03FFFF1FFCFFFFFFFFFFDF00200100F0
S11336C06A46517129680B68664A1A406B465B79F1
S11336D09B058024E403234013430593059A0A6061
S11336E002006B461A712A6814685F4B23406C46CB
S11336F02479A4068027FF043C401C430494049BC3
S1133700136003006C46E3702B681C68574F274016
S1133710BC466C46E478A4048027FF023C4067461C
S11337203C430394039C1C606C690294029CA76C48
S11337300124A743BC460700FFB23C00E407E40FA2
S113374067463C43029FBC64D520305C69460871DF
S113375028680268424911406A461279120380239C
S11337605B011A400A43049204990160D621715CFA
S11337706A46D17029684B68004A05E0FF7FFFFF65
S1133780FFFCFFFFFFFFFFF01A406B46DB78DB0313
S113379080242402234013430393039A4A60D722CC
S11337A0B25C2B685C68324F2740BC461400E4B21C
S11337B0A4038027FF013C4067463C430294029CDB
S11337C05C6000273800CC21715CC0B288422DD2E5
S11337D00020D02171583A00D2B214235A438C5A93
S11337E0220092B2D02030583900C9B21423594370
S11337F0435AD020305884463900C9B2142041437A
S1133800604640184088181882420DDA2200D2B26D
S1133810D02030583900C9B2142359434118280024
S1133820FFF7D6FC641CDBE77F1CCBE7280000F025
S113383082F92800FFF734FC002029680B680D4A40
S11338401A400300DBB2DC0580231B041C40144334
S11338500C600DB0F0BD0000FFFFFEFFFFFFFDFF99
S1133860FFEFFFFFFFFFBFFFFFFFFFFBFFFFFBFFBC
S1133870FFBFFFFFFFFF7FFF38B504000D0029786D
S113388089B22000FFF7A4FA0168C02212050A4396
S1133890026031BDF1B50C00217889B20098FFF7C0
S11338A097FA05000835217889B20098FFF7D8FA0D
S11338B000210B000A001300DBB2834238D2032339
S11338C01E00324209D129602B681600F6B2A619EF
S11338D0367A36061E432E6028E01600F6B21E40E5
S11338E0012E08D12B681600F6B2A619367A3604D2
S11338F01E432E601AE01600F6B21E40022E08D1B6
S11339002B681600F6B2A619367A36021E432E60CC
S11339100CE01600F6B23340032B07D12B681600D7
S1133920F6B2A619367A1E432E602D1D521CC2E72C
S1133930F1BDF8B506000C00217889B23000FFF71C
S113394047FA05002868000C0007000FFFF758FA33
S1133950482160542868400D0100C907C90F684612
S11339600170281D69460978002904D00168C9003E
S1133970C908616004E00168890C4905490D61606A
S1133980051D217889B23000FFF76AFA00210A0088
S11339900A000300D2B2DBB29A422AD203221300F5
S11339A0194206D12A68120E0B00DBB2E3181A7210
S11339B01DE00B00DBB21340012B06D12A68120C68
S11339C00B00DBB2E3181A7211E00B00DBB21A40F1
S11339D0022A06D12A68120A0B00DBB2E3181A7213
S11339E005E02A680B00DBB2E3181A722D1D491C8E
S11339F0CEE732689268F1BDF0B500252E000A7852
S1133A00D206D20E0124230093400F78402F12DBFC
S1133A101C0002260568002E0AD0022E04D005D30D
S1133A20032E07D12C6705E06C6703E0EC6201E02C
S1133A302C63FFE725E00E78202E11DB1D000668BD
S1133A40002C0AD0022C04D005D3032C07D13567EF
S1133A5005E0756703E0F56201E03563FFE710E018
S1133A601C000668002D0AD0022D04D005D3032DB6
S1133A7007D1346705E0746703E0F46201E034635E
S1133A80FFE7F0BDF0B50300002215000878C40676
S1133A90E40E01200600A6400F78402F16DB02201A
S1133AA01D6800280DD0022805D007D303280BD1A8
S1133AB02F6F3A0008E06F6F3A0005E0EF6A3A00B2
S1133AC002E02F6B3A00FFE732402EE00D78202D04
S1133AD015DB1D6800280DD0022805D007D3032864
S1133AE00BD12F6F3A0008E06F6F3A0005E0EF6AE0
S1133AF03A0002E02F6B3A00FFE7324015E0100075
S1133B001D6800280DD0022805D007D303280BD147
S1133B102F6F3A0008E06F6F3A0005E0EF6A3A0051
S1133B2002E02F6B3A00FFE73240002A01D0012067
S1133B3000E00020F0BDF0B5017E032937D100215B
S1133B40C9430D0002270668002F0AD0022F04D0B3
S1133B5005D3032F07D1356705E0756703E0F562E8
S1133B6001E03563FFE70A0001230468002B0AD053
S1133B70022B04D005D3032B07D1226705E062672B
S1133B8003E0E26201E02263FFE700260568002EFD
S1133B900AD0022E04D005D3032E07D1296705E0ED
S1133BA0696703E0E96201E02963FFE73EE0017E23
S1133BB0022925D10021C9430A0001250368002DEB
S1133BC00AD0022D04D005D3032D07D11A6705E0CE
S1133BD05A6703E0DA6201E01A63FFE7002604682B
S1133BE0002E0AD0022E04D005D3032E07D121675C
S1133BF005E0616703E0E16201E02163FFE715E0AE
S1133C00017E012912D10021C94300230268002B3F
S1133C100AD0022B04D005D3032B07D1116705E08A
S1133C20516703E0D16201E01163FFE7F0BDF0B535
S1133C3000231E000A78D406E40E01221500A540D4
S1133C400F78402F1ADB2A0002230668002B10D0BD
S1133C50022B06D009D3032B0FD1B76E1743B766D7
S1133C600BE0F76E1743F76607E0776A174377624E
S1133C7003E0B76A1743B762FFE735E00E78202EFA
S1133C8019DB2B000668002A10D0022A06D009D3BB
S1133C90032A0FD1B76E1F43B7660BE0F76E1F43BD
S1133CA0F76607E0776A1F43776203E0B76A1F434A
S1133CB0B762FFE718E02A000668002B10D0022B39
S1133CC006D009D3032B0FD1B76E1743B7660BE0A9
S1133CD0F76E1743F76607E0776A1743776203E0E6
S1133CE0B76A1743B762FFE7F0BDFFB591B000258F
S1133CF001200990012008900820019003210491DB
S1133D000222059214221092834A0F92FA229205FB
S1133D100E921BAA1278002A0DD1804A0D925E22BF
S1133D2002920C911F2107910299079A8918491C44
S1133D300B910A900CE0794A0D92262202920C9182
S1133D40072107910299079A8918491C0B910A9037
S1133D50139800F0EDF8040001260D98B04259DBE9
S1133D60129800F0E5F80500300000F0F1F80100C9
S1133D70280000F0F8F80500139800F0D9F80100C5
S1133D80280000F0F0F800F041F9009000980028B5
S1133D9003D000980A99884200DA3BE0009800F0CA
S1133DA0D7F80100280000F0DEF80700139800F0AF
S1133DB0BFF80100380000F07EF98021090400F00A
S1133DC0D3F908D8139800F0B3F80100380000F0D4
S1133DD072F9020006E0139800F0AAF8390000F026
S1133DE06AF902000B980099884211DB2000110047
S1133DF000F0BAF90CD809960098019014001098B4
S1133E000099884204DB10000F9900F0C1F901D336
S1133E10761CA2E714A8008800F08AF80E9900F036
S1133E20CAF9039001980299884201DA0198029034
S1133E30029C0C98844225DB2000401C38494843EE
S1133E400199FEF74FFF050014A80088281A0128DD
S1133E5003DB14A800882F1A02E014A80088471B6B
S1133E6014A8008885420DDB380000F071F803992E
S1133E7000F08EF904D20494380000F069F803903D
S1133E80641ED6E701980499401A401E05902548FF
S1133E90039001250598A84221DB21486843019934
S1133EA0FEF720FF07001AA80088381A012804DB4F
S1133EB01AA80088381A069003E01AA80088C01BC4
S1133EC00690069800F044F8039900F061F904D2D2
S1133ED00895069800F03CF803906D1CDAE7099801
S1133EE011990860049800F0CFF90FA20CCA00F0F1
S1133EF0D5F900F095FA11998860049811998968A8
S1133F00401A1199C8600598119908610898119987
S1133F10486015B0F0BD0000CDCCCC3DFF030000DF
S1133F201027000000401C46333333333333E33F60
S1133F309D2102000AD002D4491E9218FCD5C9055D
S1133F40100A1206524100D3012A4841704700006A
S1133F509D210200EED55242F446FFF7EBFF012209
S1133F60D2071043604730B405004D400122D20708
S1133F7015404B180418240E25D01B0E2CD0FF2CF2
S1133F8031D0FF2B34D0E41A00020902104311434C
S1133F9043084808D10D1B1A02D2641EDB181B18F3
S1133FA0DB18834200D31B1A4941F9D37F3423DD44
S1133FB0FF2C05DAE40548086041284330BC70470B
S1133FC0FF20C005F9E728001B0E03D0FF2BF5D115
S1133FD04902F3D0D043F1E7FF2C01D14002F9D1DB
S1133FE0FF20C005E9E74002F4D1FF2BF8D1F1E747
S1133FF028004902E2D0EDE70B0200202442DCD184
S11340005B129B1CD9D9D805D7E7FEE70122D2075A
S11340100118090E7F3910D449421F310FD40018FA
S113402005D2C0011043C84000D5D0437047C00139
S11340301043C84005D440427047002070470042F6
S1134040F3D5100070470122D20703004B402ED451
S1134050431A01D2C01AC91830B44B180418240EDC
S11340601B0E22D0FF2C20D0E31A182B1DDC0902D2
S11340701143C40D641E0002104394461925ED1A21
S11340800A00AA40D940451801D36D08A41CE405D0
S1134090D209280A2D062A436546AA41604103181D
S11340A01B0EFF2B01D3C00DC00530BC704751401F
S11340B006E05140CCE70122D20703004B40F8D47C
S11340C0431A03D2C01AC9185040514030B44B1897
S11340D0090211430418240E1B0E40D0FF2C3AD0C1
S11340E025009D410BD31ED8C50D4002401A0BD3A9
S11340F0ED050100400AC90591416841D5E7C50DA8
S113410040024918401AD0D001214008491C001827
S1134110FCD58C4204D36D1A000AED054019C4E79E
S1134120E8051040C1E7182DBFDCAC1C0D00E140D0
S1134130E5414D40012D4941C40D00021043451A8B
S113414001D46D199543641EE405280A2D06954192
S1134150604130BC7047FF2BA7D1D843A5E7244268
S1134160A3D10020A1E7FEE70CB401221206031834
S1134170DA4207D84B18DA4204D802000A439218EC
S113418002D281420CBC7047FCD088420CBC704700
S11341900CB4012212060318DA4207D84B18DA428B
S11341A004D802000A43921802D288420CBC704719
S11341B0FCD08142FAE730B405004D400122D20719
S11341C015404B180418240E2ED01B0E32D0FF2C91
S11341D034D0FF2B3AD0E4180002090210431143F3
S11341E0000A090A9446C2B24A43000AC3B24B43C6
S11341F0000A4843110A5B181A43D2B2190A091873
S113420001D44918641E080A7F3C23DBFE2C08DA1B
S1134210E40509061143634699416041284330BCD3
S11342207047FF20C005F9E728001B0EFF2BF6D1CD
S1134230D043F4E72800FF2CF1D1F9E74002F7D18D
S1134240FF2B01D14902F3D1E005E7E7D805490284
S1134250E4D0EDE743020020641CDFD15B129B1C19
S1134260DCD9D805DAE7FEE7010042221201D21EAA
S1134270004207D002D4521E0018FCD5C10A4005E2
S113428012058918704700000100EED54042F4463B
S1134290FFF7EBFF0122D20711436047F0B50E0090
S11342A05E400125ED072E40B446AE0ADF184C18D7
S11342B0F44208D2F7420ED2640D01D07F0D12D120
S11342C000206146F0BD05D1F74201D87F0D05D12C
S11342D00020C143F0BDFBD1640DF9D00020C143DF
S11342E0490549088FE0E419C902DB0229432B433D
S11342F0DB0A460DC00231438E4630B487B295B214
S11343007D432E0CADB2140C7C43A419260C24045A
S113431025439CB27C43A419190C7943270CC91971
S1134320A4B20F043C43090C000C97B247432E0C73
S1134330BE193543ADB2170C4743360CBF19A6B2AC
S1134340BF193E043543240C3E0C36199FB2474333
S1134350BF19BCB23E0C89191F0C47437F183E0499
S11343603443390C704680B297B247432E0CBE19C1
S11343703543ADB2170C4743360CBF19A6B2BF196B
S11343803E043543240C3E0C36199FB24743BF19F3
S1134390BCB23E0C89191F0C47437F183E043443BA
S11343A0390C77463F0C90B278432E0C80190604E2
S11343B0ADB22E43050CA0B22D18120C7A4350193D
S11343C0020C80B2240CA4189AB27A431219140471
S11343D02043120C89181B0C7B43C91830BCEF0A0C
S11343E0394203D1B61940414941641E6F12BF0DD1
S11343F0E41B0BDBFF19BC4211DA24050027420839
S1134400AE417841614166463143F0BD641C05D13B
S1134410401C6141CF0201D34908F4E750E75DE74E
S11344204A1812D2400DC90208430121C9070843A2
S1134430520D40210901521A521C06D452421F3215
S113444001D4D0407047C017704700207047000067
S1134450F8B59CB0050000263700300069460870A6
S1134460029601963400300069468870402200218B
S11344700CA800F00DFE04A8D349202200F012FE7F
S1134480082069464870FF20801C0390300001001A
S11344906A465278C9B291420FD20021C9430CAA8C
S11344A00300DBB2DB00D15031000CAA0300DBB205
S11344B0DB00D2189180401CE9E7370038006946D8
S11344C04978C0B288424BD20220040003982100EC
S11344D089B288423ED3286804A93A00D2B2920035
S11344E08958FEF702FC210089B2FEF7FEFB019019
S11344F001986968884213D10CA83900C9B2C9006F
S113450041188C803900C9B2C900401887710CA8C1
S11345103900C9B2C900465001206946887019E0C3
S113452001986968884213D20CA83900C9B2C9003D
S113453041188C803900C9B2C90040188771686875
S11345400199401A0CA93A00D2B2D200885001E075
S1134550641CBBE768468078002801D17F1CADE766
S1134560684606700CA869460978C900405802904C
S11345700126300069464978C0B2884211D20CA89D
S11345803100C9B2C90040580299884207D20CA828
S11345903100C9B2C9004058029068460670761CC2
S11345A0E7E70CA869460978C900411889880229F7
S11345B017DA286804A96A46527892008918091FF4
S11345C00968FEF792FB0399FEF78FFB019068469A
S11345D04078401EA8600398801EE8600198286116
S11345E014E069460978C90041188979A9606946C7
S11345F00978C90040188088801EE86068680CA9A2
S11346006A461278D2008958401A28611DB0F0BD5C
S1134610F8B58AB004000D00002000900700029055
S11346202000006E00900021684600F0F4FC002198
S1134630684600F0E1FC697B684600F0A3FC697AF7
S1134640684600F075FCA97A684600F068FC686862
S113465006902868059005A8FFF7FAFE07986946B2
S1134660087108980290029E03940398006CFF213D
S113467088433100C9B20143049104980399086442
S113468068460179684600F061FCE989491E89B2EF
S1134690684600F0F3FCA87B800604D5E97E6846F2
S11346A000F07EFC03E00021684600F079FCE97A22
S11346B0684600F059FC687D002805D0022829D0FE
S11346C010D303283ED04BE00021684600F0B2FC32
S11346D0E97F684600F090FC2020295C684600F0E1
S11346E09AFC4AE00121684600F086FC00216846F5
S11346F000F091FC287C002804D10021684600F0D9
S113470099FC06E0287C012803D10121684600F0C9
S113471091FC32E0287C002804D10021684600F096
S113472089FC06E0287C012803D10121684600F0B9
S113473081FC0121684600F05FFC0021684600F01E
S11347406AFC1AE00021684600F074FCE97F6846C0
S113475000F052FC2020295C684600F05CFC0CE070
S11347600021684600F066FCE97F684600F044FCDE
S11347702020295C684600F04EFC009820660BB0AF
S1134780F0BDF8B50A7A6B461A700200536A6C469B
S11347902478012C03D101241C43546202E05C08F8
S11347A0640054620C7BCD7AAC4005006E6ACB4F3A
S11347B03740BC462600F6B23702F02636013E40AA
S11347C067463E436E62F1BD08C40000F6B588B08A
S11347D0099909780200D6690B00DBB2012B03D1D9
S11347E001233343D36102E073085B00D361099B67
S11347F05B780400E5691F00FFB2012F03D1022199
S11348002943E16103E0290002229143E16109990E
S113481089780200566A0F00FFB2012F03D10823E2
S11348203343536203E033000824A3435362099BD8
S1134830DB780400256A1F00FFB2012F04D1802118
S113484049002943216202E0A549294021620090E0
S113485000210E000122009F7F6A1740002F01D023
S113486013001E00F6B2002E0FD1099B5B790400E1
S1134870656A1E00F6B2012E03D104262E43666239
S113488003E02E000427BE436662099BDB796C4675
S1134890237005002E696B461B78012B03D104237A
S11348A033432B6103E033000424A3432B61099BAE
S11348B09B796C46237103001C696F463F79012F75
S11348C003D1082525431D6103E025000826B543CF
S11348D01D61089D6D786E46F5700490049D2E6CE4
S11348E0804D35406E46F67836022E430796079D76
S11348F0049E3564089DAD786E46B5700390039DA3
S11349002E6C794D35406E46B67836042E430696A5
S1134910069D039E3564089DED786E467570029081
S1134920029D2D6C2D022D0A6E46767836062E4396
S11349300596059D029E3564089D2D796E46357059
S113494005006F6A7026B743BC466E463678370159
S113495070263E4067463E436E62089F7F79002F73
S113496005D0022F39D024D3032F4AD06DE0089B01
S11349709B79002B00D10A0003005C6A1500EDB29C
S1134980002D04D08025ED0425435D6202E0574DDF
S113499025405D6205006E6A554F3740BC460E00E7
S11349A0F6B23706C026B6043E4067463E436E6202
S11349B06CE013000400616A4D4D0D401900C9B24A
S11349C00E06C021890431402943616205006E6AE4
S11349D08027FF0437436F6258E002230400616AB2
S11349E0434D0D401900C9B20E06C021890431405F
S11349F02943616205006E6A8027FF0437436F62B2
S1134A0044E0089B9B79002B01D01100FFE70200D2
S1134A10536A0C00E4B2002C04D08024E4041C4348
S1134A20546202E0314C1C405462032405006E6A57
S1134A302F4F3740BC462600F6B23706C026B604D0
S1134A403E4067463E436E6220E0089B9B79002B04
S1134A5000D10A0003005C6A1500EDB2002D04D0F9
S1134A608025ED0425435D6202E0204D25405D6212
S1134A7005006E6A1E4F3740BC460E00F6B237067C
S1134A80C026B6043E4067463E436E620AB0F0BD9F
S1134A908149016081494160012202720021417211
S1134AA08172C172017342730822C281C175017699
S1134AB041768176C17601774177C177202281548E
S1134AC08177022202740A22130043741300837450
S1134AD0C27401754175817570470000FFF0FFFFD6
S1134AE0FFFEFFFFFF00FFFFFFFF00FFFFFFFFFBD5
S1134AF0FFFFFFFCF0B587B004000D0000206946FD
S1134B004870206802900298006906900698012176
S1134B108843029908612068019001980069059012
S1134B20059880214900014301980161276838698B
S1134B3004900498802189000143396100BF00BFBB
S1134B4000BF29002068FFF71CFE2A001732290045
S1134B5010312068FFF73AFE012001006A46117007
S1134B60266831690391039908433061290020685C
S1134B70FFF74EFD07B0F0BDF2B482B002990160B8
S1134B8001680A690192019A80235B0013430B6157
S1134B90026813690093009B8024A4001C431461E1
S1134BA001230468256902262E43266100BF00BF45
S1134BB000BF002607683E61F7BC7047F0B50300EC
S1134BC00022100014000D006D1E17D06D1E1DD0A4
S1134BD0FE3D24D080267600AD1B29D08026B60069
S1134BE0AD1B2ED08026F600AD1B33D080263601B7
S1134BF0AD1B38D08B4EAD1B3ED046E01D686F69AF
S1134C003E00F607F60FF6B234003EE01D686E690A
S1134C1077083E00F607F60FF6B2340035E01D685B
S1134C206E69370A3E00F607F60FF6B234002CE040
S1134C301D686E69770A3E00F607F60FF6B2340077
S1134C4023E01D686E69B70A3E00F607F60FF6B258
S1134C5034001AE01D686E69F70A3E00F607F60F85
S1134C60F6B2340011E01D686E69370B3E00F6079A
S1134C70F60FF6B2340008E01D686E69370E3E0088
S1134C80F607F60FF6B23400FFE7002C01D001223C
S1134C901000C0B2F0BD000000B4C40440420F00D4
S1134CA0FFB583B0012069460870002420000399F1
S1134CB009682200CB6DDB06DB0E1025EB1A6D466E
S1134CC06B706B465B786D46AD8A9BB2AB4200D28B
S1134CD0A2E00194250020006946488003980068FA
S1134CE0006E0190002101A800F078F9012101A8CB
S1134CF000F065F9002101A800F08DF9002101A858
S1134D0000F07AF96846007CC100491E89B201A806
S1134D1000F0B4F901980399096808662600300088
S1134D206946898A80B2884269D203980168220060
S1134D3001204F6903003B40DBB2002B06D16D1C00
S1134D4039498D42F1D321006A4611706946097CC4
S1134D50012907D10699320092B2895C039A12683C
S1134D60516614E06946097C022908D1069932008B
S1134D7092B25200895A039A1268516607E0069962
S1134D80320092B292008958039A12685166250043
S1134D900399096822000B6F5B080340002B01D0C4
S1134DA003001A00D2B2002A06D06D1C1E498D429F
S1134DB0EED32000694608706846007C012807D1BC
S1134DC003980068406F0C99320092B2885414E042
S1134DD06846007C022808D103980068406F0C994B
S1134DE0320092B25200885207E003980068406F84
S1134DF00C99320092B292008850761C8FE7002101
S1134E0001A800F0EBF8002101A800F0D8F80198FF
S1134E1003990968086601E06846047068460078EA
S1134E2007B0F0BD00F0FF00E9030000F0B5030097
S1134E30002210000C00641E14D0641E1CD0FE3C22
S1134E4024D080256D00641B2BD08025AD00641B0D
S1134E5032D08025ED00641B39D080252D01641BE0
S1134E6040D04AE0012425001E68B7692F40AF42B4
S1134E7000D12200100040E002241D68AE692640E3
S1134E80A64201D101263200100036E080246400DD
S1134E901D68AE692640A64201D1012632001000E9
S1134EA02BE08024A4001D68AE692640A64201D1EF
S1134EB001263200100020E08024E4001D68AE6961
S1134EC02640A64201D101263200100015E08024BC
S1134ED024011D68AE692640A64201D10126320094
S1134EE010000AE0802464011D68AE692640A642D1
S1134EF001D1012632001000FFE7C0B2F0BD70B44A
S1134F000A0003689D6D524C2C401500EDB22E042E
S1134F10F8256D03354025439D6570BC70470268D4
S1134F20520052080B00DBB2DB07134303607047E7
S1134F3010B40268474B13400A00D2B2920780248F
S1134F40E40522401A43026010BC704710B40268A2
S1134F50414B13400A00D2B2D406E022920522400B
S1134F601A43026010BC704710B402683B4B1340F4
S1134F700A00D2B21406C022920422401A430260EC
S1134F8010BC704710B40268354B13400A00D2B20B
S1134F90D2058024240422401A43026010BC7047C6
S1134FA000B502680B00DBB2012B04D18023DB03C4
S1134FB01343036002E02B4B1340036000BD00B5B4
S1134FC002680B00DBB2012B04D180239B03134343
S1134FD0036002E0244B1340036000BD10B4026878
S1134FE0224B13400A00D2B21205802464032240EB
S1134FF01A43026010BC704700B502680B00DBB2B4
S1135000012B04D180231B031343036002E0184BDC
S11350101340036000BD00B502680B00DBB2012B36
S113502004D18023DB021343036002E0114B1340DD
S1135030036000BD10B402680F4B13400A00D2B2E3
S11350401404C022920222401A43026010BC70472A
S1135050FFFFE0FFFFFFFFBFFFFFFFC7FFFFFFFCF6
S1135060FFFF7FFFFFFFBFFFFFFFDFFFFFFFEFFF3C
S1135070FFFFF7FFFFFFFBFFFFFFFCFF0268120BC0
S113508012030B009BB21B051B0D134303607047F7
S113509010B50400080011000200200000F02AF8F6
S11350A0200010BD70B4103A03D378C9103A78C008
S11350B0FBD2530701D318C918C001D508C908C0C9
S11350C0D20704D30B880380891C801C002A01D5D5
S11350D00B78037070BC70478B0701D18307E1D054
S11350E0124205D00B78491C0370401C521EF9D1A2
S11350F0704700001206130A1A43130C1A4300BF28
S1135100094205D0830705D00270401C491EF9D11D
S1135110704700001300103906D330B41400150092
S113512010393CC0FCD230BC490700D30CC000D5B8
S113513004C0890002D30280801C002900D50270BB
S11351407047000000B5010008000200D2B2802AB6
S113515001DB7F221000C0B200BD00B501000800D1
S1135160C0B2F12805DB0800C0B2FA2801DA012038
S113517006E00800C0B2802801DA080000E0002040
S1135180C0B200BDFEB582B0070000252C006E46FB
S11351903F20307030786946097AF0220A43024091
S11351A032706846007B70706846007CFFF7CAFF67
S11351B0B0703878002810D0032004002000C0B25A
S11351C0082804DA2000C0B23554641CF6E708222B
S11351D06946F868BB6D984704E003226946F8689D
S11351E0BB6D984740B205B0F0BDFEB50600002087
S11351F0050001006A460F2313701378F48AF02720
S113520027431F40177004002100C9B2F38A89B2F2
S1135210994209D231692300DBB2C95C2300DBB2B5
S1135220D3185970641CEFE73178002916D00500B3
S11352302800C0B20721F38AC91A884208DA280074
S1135240C0B2F18A40181018CC2141706D1CEFE7F0
S113525008226946F068B36D984706E0F28A521C4A
S1135260D2B26946F068B36D984740B2FEBD3EB510
S1135270050068461F2101700178EA8A92B2120A79
S1135280F02313430B400370E98A4170002421008A
S1135290C9B2E4B22100C9B2062909DA2969220097
S11352A0D2B2895C2200D2B282189170641CF1E7F8
S11352B008226946E868AB6D9847010049B20029A5
S11352C004D1298B891D29830121A97640B23EBDD1
S11352D0FEB5060000273900C9B201A82F220270CA
S11352E00278B37EF0241C4314400470F28A338B9A
S11352F0D21A6B461A806A461288082A02DB0722F1
S11353006B461A803C00E4B22100C9B26A46128896
S113531089B291420BD23169328B2300DBB2D218AD
S1135320895C2200D2B282185170641CECE7317897
S113533000291BD03900C9B23D00EDB22A00D2B217
S113534007216B461B88C91A8A4209DA2900C9B2A7
S11353506A46128889184118CC224A706D1CEDE700
S1135360082201A9F068B36D984707E068460288EF
S1135370521CD2B201A9F068B36D9847010049B23A
S113538000290BD1318B6A46128889183183B17E8A
S1135390491CB176B17E102900DBB77640B2FEBD60
S11353A0F8B504000D00160000210F000F202B7823
S11353B00200134206D03200D2B2521E2B780340B0
S11353C09A4208DA606D002802D0A248616D8847CD
S11353D00620C04315E02A7810404222A05208005B
S11353E0C0B24222A25A80B2904209D20800C0B28E
S11353F028184078E26B0B00DBB2D054491CEEE76E
S11354000020F2BDF8B504000D00170000210800CB
S11354106A4610703800C0B2082808D0606D0028B1
S113542002D08D48616D88470620C04339E0287852
S11354300002F0221201024068781618300080B28F
S1135440082808DA606D002802D08448616D884716
S11354500620C04325E04020205A320092B29042F8
S113546008D2606D002802D07D48616D8847022013
S1135470C04316E0422026520800C0B2062809DACA
S11354800800C0B228188078E26B0B00DBB2D0545D
S1135490491CF1E706204422A05201204622A054D0
S11354A00020F2BDF4B505000C00002217004620D0
S11354B0285C21780907090F884202D00320C043E1
S11354C040E04220285A4421695A461A300080B2EA
S11354D0082801DB0720060068460078401E3100DA
S11354E089B2884208DA686D002802D05D48696D87
S11354F088470620C04325E011000800C0B23300ED
S113550080B29BB298420CD2E86B0B00DBB244270A
S1135510EF5BDB190F00FFB2E7197F78C754491C12
S1135520EBE74420285A80194423E8524620285C9B
S1135530401C4623E8544620285C102801DB462002
S11355402A540020F2BD70B504000D00160030008E
S1135550C0B2032808DA606D002802D04248616DA9
S113556088470620C04300E0002070BD70B50400E9
S11355700E0015002B009BB23200E168200000F001
S113558001F870BDFEB5040000263700002C02D1DE
S11355900020C0435CE0A08A69460989884208D299
S11355A0606D002802D03148616D88470220C043F5
S11355B04EE03420205C012808D1606D002802D020
S11355C0CA48616D88470120C04341E068460089AC
S11355D0E0823000208335002800C0B26946098982
S11355E080B2884209D201982900C9B2405C21697D
S11355F02A00D2B288546D1CEEE7E08A082804DA47
S11356002000FFF7F2FD070020E02000FFF72FFE47
S11356100700380040B2002818D13000A0833000C1
S1135620A0773000E077E06D80472200203203C28B
S1135630083AE06D8047002264305141220028324C
S113564003C2083A2663012034216054380040B272
S1135650FEBD000070C300009CC3000068C20000CF
S1135660A0C20000C8C30000E8C30000D8C2000004
S1135670FFB583B004006846007E022803DB684659
S1135680007E092800DB2FE100252900C9B228008B
S1135690C0B201006A46127EC9B2914209D205998C
S11356A00200D2B2895C01AA0300DBB2D154401CCF
S11356B0EFE72F00FFB23800C0B208216A46127E1D
S11356C0891A884208DA01A83900C9B26A46127EEA
S11356D0891845547F1CEEE701AE3078C0B200094A
S11356E0002806D0022865D021D3032800D1B3E0D6
S11356F0FAE05120205C012804D10520C043502148
S1135700605401E0502025546846027E01A920001F
S1135710FFF746FE694608706946002008560028CF
S113572004D10498A063022051216054DCE051208C
S1135730205C012804D10520C0435021605401E0BD
S1135740502025546846027E01A92000FFF75AFE26
S1135750694608706946002008560221C9438842F8
S11357600CD10720C04350216054512025540023FC
S1135770002202212000FFF705FDB5E06946002064
S11357800856002815D10498A063012051216054C3
S113579060784721605401234720225C00212000C7
S11357A0FFF7F0FCE06D8047002264305141A064B3
S11357B0E16499E05120205C012804D00520C04315
S11357C05021605490E00498A16B884200D08BE093
S11357D06846027E01A92000FFF764FE694608704E
S11357E00326F643694600200856B04207D101A8B3
S11357F000F0A6FB502026545120255474E069463D
S113580000200856002826D1E06D8047002264302D
S11358105141A064E1644420205A4221615A8842E3
S113582003D302205121605415E06078002812D07F
S11358304720205C401E472160544720205C0028FC
S113584009D160784721605401234720225C00215C
S11358502000FFF797FC47E03420205C012843D167
S11358606846027E01A92000FFF76DFE69460870B4
S1135870694600200856002835D1E06D8047002293
S1135880643051412200283203C2083A0F20317893
S11358900140022906D10720C0432063022034219D
S11358A0605420E03178014001290CD1E07F401C94
S11358B0E077E07F022816DB0620C0432063022045
S11358C0342160540FE0317801420CD17078002803
S11358D002D18448A08301E07078A083B078FFF7F8
S11358E03CFCA077E577FFE707B0F0BD0CC30000F0
S11358F0FEB50100089A0020030051240C5D022C1F
S113590002D00420C04328E08C6B8D68AC4201D1E6
S1135910012400E00400009D2C7042240C5B6D46C1
S11359202D892600B6B2B54202D26D462D892C00CF
S113593005002B0026009BB2B6B2B34209D2CB6B52
S11359402E00B6B29B5D019E2F00BFB2F3556D1CB5
S1135950EFE714805123C8540020FEBD70B4020048
S11359600B00187810705878507058685060986818
S11359709060D868D06018691061988A9082002479
S11359802000D08220001083200090762000908395
S1135990200090772000D0770020002115002035CA
S11359A003C5083D1500283503C5083D14632500CB
S11359B0342695559D69D5639D8B402695532500C6
S11359C04226955325004426955325004626955591
S11359D02500472695559064D164200050215054E9
S11359E051201454186A5065586A9065986AD065B5
S11359F070BC704770B504003420205C01285AD173
S1135A00384DA08BA84202D0A08B002841D0A07FA3
S1135A10002810D0A07F00283BD0E06D8047020012
S1135A200B002000203003C8801A9941002930DC83
S1135A3001DB00282DD22000FFF74AFC06003000CD
S1135A4040B2002822D1A08BA84202D0A08B4019DA
S1135A50A083E06D80470022643051412200283247
S1135A6003C2083AE06D804702000B00A07F0021CA
S1135A70801859412200203203C2083A208BE18A5F
S1135A80884206D300203421605402E002203421ED
S1135A906054E06D8047220028320CCA121A8B41F0
S1135AA0002B08DC01DB002A05D20120C04320635F
S1135AB00220342160545120205C012811D1E06D72
S1135AC08047A26CE36C121A8B41002B09DC01DBCA
S1135AD0002A06D20220C0435021605400205121E4
S1135AE0605470BDFFFF000008B4024B9C4608BC24
S1135AF06047C04639020020F0B5020052B2002AC5
S1135B0017D41822B74B040064B2A408A4001C598B
S1135B10FF25C6001640B540AC438D01EDB2C6006A
S1135B20324095402543020052B2920892009D50A3
S1135B301BE00F22AC4B182405006DB21540083D44
S1135B40AD08AE0005006DB22A40083A92089200F2
S1135B509A58FF25C7002740BD40AA438D01EDB2E6
S1135B60C7003C40A54015439D51F0BD10B504004D
S1135B70601E80214904884201D301200EE0601E8A
S1135B809A49086003210020C043FFF7B5FF0020B5
S1135B90974908600720BD490860002010BD002215
S1135BA002604160012303724272704700B5017ABA
S1135BB000290FD0417A00290CD101684268914232
S1135BC008D20168491C016001684268914201D110
S1135BD00121417200BD70B504000E001500AC48EF
S1135BE0215AD6482018FFF7DAFF7820205C0128D4
S1135BF006D02A0092B2310020001830FFF7B6FC1C
S1135C0070BDFEB505000E001400082100226F4689
S1135C103800FFF76FFA2000C0B2782805D09C48FE
S1135C20295AC6482818FFF7BAFF7920285C0028AB
S1135C3014D02000C0B211280FD02000C0B2122806
S1135C400BD02000C0B2312807D02000C0B27E287B
S1135C5003D02000C0B27F2800D10AE068467F212B
S1135C600170467084700322694628001830FFF7DB
S1135C707DFCF7BD10B5040088200001201803C87E
S1135C800022401C514188221201A21803C2083A82
S1135C90892000012018FFF789FFB5482018FFF775
S1135CA085FFA6482018FFF781FF10BDB14803C83F
S1135CB0704780B5B0480168491C0160AD4A03CA09
S1135CC0083A0023401C594103C2083AC448FFF76C
S1135CD0D1FF01BDF8B596B0002000216A461170CD
S1135CE0C04C68460078CC21615C884251D2684639
S1135CF0007869460873BC4D03A92868FDF7C2FE05
S1135D00002840D0D02020586946097814225143F5
S1135D104018407A012832D103A92868FDF76CFEA7
S1135D2003A92868FDF705FE03AC4820205C029017
S1135D3003A808300190AD4D982040012E1830780A
S1135D404C2148432818071D029A01993800FFF78F
S1135D50C3F9049831784C225143685030784C216F
S1135D604843281844214822A25C42543078401CFD
S1135D7030703078202806D30020307003E003A967
S1135D802868FDF739FE68460078401C69460870AB
S1135D90A6E717B0F0BDF1B582B0002468460470E0
S1135DA092489349451898214901415C2A789142C7
S1135DB015D04C2629784C22514340180190029F5B
S1135DC0320001993800FFF787F92878401C2870C1
S1135DD02878202800D32C70012069460870684672
S1135DE00078FEBD00E400E01CED00E014E000E0FB
S1135DF018E000E0F3B595B0170000242600F6B2D1
S1135E002000C0B2E4B277482100CC22825CC9B23F
S1135E1091420ED21599D02282582300DBB2142568
S1135E206B43D2185268914201D1260001E0641CF0
S1135E30E9E7D03002A902683300DBB214256B43D2
S1135E40D25A0A7048228F5400683100C9B2142211
S1135E5051434018406803903800C0B2019016982E
S1135E60009002A805000835019A00992800FFF760
S1135E7033F95D4D02A92868FDF70CFD02A92868D5
S1135E80FDF7FAFC002017B0F0BD000010E000E0C0
S1135E908C080000FEB500240294534F554E300088
S1135EA0803038603500D03505220021280000F00C
S1135EB036FA05220121280000F031FA494D280064
S1135EC0FDF79BF80420CC2168544B48D02168503E
S1135ED0012001002970210069702100A9702100AE
S1135EE0E97030216C54C821685402AA0B21300097
S1135EF00830FCF776FE687801280BD10120019068
S1135F00FA20C0000090A94BA94A029928001C302D
S1135F10FDF7EBFE00200190A6480090A34BA64A93
S1135F20029928000830FDF7E0FE29003868FDF7E3
S1135F3085F9092000F082FAF7BD0000A8080000E6
S1135F4010B5040000200100C9B2082908DA0100D4
S1135F50C9B2615C994A0300DBB2D154401CF2E738
S1135F60082296498D208000FFF744FF10BD0000F1
S1135F709C08000000200020A0320020F8B586B064
S1135F80012501AC28002070022630006070280032
S1135F90A0808B4F01AA07213800FCF73FFE2800A0
S1135FA0207030006070A68001AA07213800FCF739
S1135FB035FE25700720607001AA29213800FCF7FE
S1135FC02DFE8048006E009002216846FEF7BEFF59
S1135FD000F03CFA00F0B9FB07B0F0BD000000008F
S1135FE008200020D04F0020A8500020CC3C0020E6
S1135FF0011300001C310020C8C10000F8B59CB09A
S113600000F064FD7049002000F0BCFF00F00CFAC1
S11360106E4C200000F0C6FFC0204000201801F0A4
S11360205FF86B480390002002906A4D029A03992E
S11360302800FFF75FF8D820019000200090664DFB
S1136040009A01992800FFF755F804A8012101706E
S11360500121818004AA132120000830FCF7DEFD11
S113606004AA142120000830FCF7D8FD04AA152145
S113607020000830FCF7D2FD04AA162120000830C5
S1136080FCF7CCFD04AA172120000830FCF7C6FD5C
S11360902500E03501220121280000F040F900220A
S11360A00121280000F096F902220121280000F0C5
S11360B0B6F8FFF7EFFE494F4949380001F03AF8C6
S11360C0484E494B494A3900300001F0BAFA484D6C
S11360D02A00092120000830FCF783FD2868FA21F2
S11360E08900FCF702FEFFF741FD424800F0A6F9E3
S11360F03000FFF7F9FC00F089F93F4801680029F6
S11361003DD0002404603D4D2868401C2860286868
S11361100A21FCF7EAFD002905D139480078012855
S113612001D100F0ABFA2868FA21890088420FD324
S11361302C60012000F0B0FA04003248026811001B
S1136140491C01602300DBB22F49002000F01AFF34
S11361502B48017800290AD12C490A78521C0A706C
S113616009780B2903DB01210170FFF707FF0120E8
S113617001F06AFB380001F041FC01F04FFB09A873
S1136180FFF709FE0128B8D109982149884203D0B4
S1136190099820498842B0D109A84421435C021DD2
S11361A0099938001830FFF763FAA6E74C1D000080
S11361B080841E00C409000020A10700EC06002012
S11361C02431002080320020A8C400001C310020AB
S11361D004130000CC3C0020D04F002008200020F5
S11361E0B80600207C310020035C0000D75B00006F
S11361F0A8320020FFFF0000A0320020A4320020BB
S1136200D3550020AC500020C0C40000D25500205B
S113621031070000DF070000016042607047F5B5F8
S113622083B0122979D26846007C002803D0022862
S11362304DD026D371E00023684643700800039ACA
S11362401268840014590225AC436D466D786D00C4
S11362500226354025430195019C850054516C4626
S113626023700B00039C24689D0065590126B543E7
S11362706E4637783E00F607F60F2E439D006651B2
S11362804BE0012002000191039B1B68019CA400C8
S11362901C590225AC431500EDB26D0002263540B1
S11362A025430295029C019DAD005C5100240091A0
S11362B0039D2D68009EB600AE590127BE432700FA
S11362C0FFB238403043009EB600A85125E00020BC
S11362D00191039A1268019B9B00D3580224A343A3
S11362E00400E4B2640002252C401C430294029B87
S11362F0019CA400135101231C000091039D2D68EF
S1136300009EB600AE590127BE432700FFB23B40B2
S11363103343009EB600AB51FFE705B0F0BDF5B5C1
S113632082B06846007B002828D16846007B6A4614
S113633010700800029A12688300D458244B23403A
S11363406C4624782402E025ED0025401D43019588
S1136350019B8400135101230C00029D2D68A600AB
S1136360AF590426B743BC461E00F6B2B600042754
S11363703E4067463E43A700EE5127E000200A0056
S1136380029B1B6894001C590425AC430500EDB224
S1136390AD000426354025430195019C95005C51D0
S11363A06C46247B6D462C700C00029D2D68A60063
S11363B0AE59074F3740BC466E4636783702E02662
S11363C0F6003E4067463E43A700EE51FFBD000085
S11363D0FFF8FFFF30B443685B6901248C40A3439A
S11363E01400E4B28C401C43230045686B6130BC4C
S11363F07047000000B5010049B2002905D401210D
S1136400C206D20E91400B4A116000BD00B50A4885
S11364100168012906DB0168491E01600068012842
S113642000DA62B600BD000072B603480168491C78
S11364300160704700E100E01831002010B504004D
S1136440200040B2FFF7D6FF10BD000018B589B098
S113645000F041F86846FEF71BFB0120694608720C
S1136460804A0192C87248727F4C6A4629212000F2
S11364700830FCF7B6FB0028F6D0B2204000241800
S113648069462000FEF736FB00212000FEF737FDA9
S113649000200AB010BD7CB506000D00734B1E70C1
S11364A05D70734C0094022201217248FEF7F8FBE0
S11364B0207800026178084380B276BD10B56D4C37
S11364C002212000FEF77AFB012803D102212000DB
S11364D0FEF7ACFC10BDF0B595B0674C0322052166
S11364E02000FFF71CFF01256846C57105200E90AA
S11364F021680D910D990E9A92008958402291437A
S11365006A46D279920140231A400A43149214999C
S11365100D9A0E9B9B00D15069468D710C9020689A
S11365200B900B980C99890040582027FF43384062
S11365302026694689794901314001431391139812
S11365400B990C9A92008850032202212000FFF735
S1136550E6FE6846457102200A902168099109996E
S11365600A9A92008958402291436A4652799201CC
S113657040231A400A431292129B09990A9A9200E4
S11365808B5069460D710890206807900798089908
S1136590890040583840694609794901314001432E
S11365A0119111980799089A9200885003220421A6
S11365B02000FFF7B4FE6846C570042006902168E9
S11365C005910599069A92008958402291436A469A
S11365D0D278920140231A400A431092109B0599E5
S11365E0069A92008B5069468D700490206803903F
S11365F003980499890040583840694689784901CC
S1136600314001430F910F980399049A92008850E6
S1136610032203212000FFF782FE68464570032011
S113662002902168029A92008B58402293439C4620
S11366306A465278920140231A4063461A43029BE9
S11366409B00CA506B461D70236884001C59274068
S11366506C462478640126403E4384001E5115B0E4
S1136660F0BD000040420F001C310020685500209E
S11366707455002080320020EC3100201CB503202A
S113668000F00AF8040000222100C9B2032000F03F
S11366900BF80090009816BD10B5040000216006A8
S11366A0400EFFF7F8FE10BDF8B505000C0017000A
S11366B02100C9B280202843C0B2FFF7ECFE0600D7
S11366C0002F00D03E80684605702800C0B2FFF756
S11366D0E3FF604069464870684684700098F2BDE4
S11366E0FEB582B004000F000A9E2000C0B2FFF77E
S11366F0D3FF0500002E00D035802800B84369463A
S1136700097C6A46127B91400143684601706846E1
S1136710017880202043C0B2FFF7BDFE68460471B3
S11367206846007C6946097B884001A9887020007E
S1136730C0B2FFF7B1FF0100394001A8807848409A
S113674001AA5070019805B0F0BDF0B599B01527B5
S11367503800002529006A4651710100C9B20909AF
S113676041400800C0B2800848400100C9B249084D
S1136770414068460171684600790100C907C90FA4
S1136780012901DB952007002C000495200080B22C
S1136790C008694648732000400169460873280010
S11367A06946C8722800694688720498C008694618
S11367B04872049840016946087228006946C87105
S11367C028006946887105A832495022FEF76AFC00
S11367D005AE77706846407B292170546846007B7B
S11367E02B2170546846C07A2D2170546846807AF3
S11367F02F2170546846407A312170546846007ADB
S1136800332170546846C0793521705468468079C4
S113681037217054684640794B217054FFF716FEB7
S1136820002809D0280069460870FF20694648708E
S11368306846857000982BE02C002000C0B2400010
S1136840305C002806D12000C0B2400030184078E7
S1136850002814D000222000C0B240003018417833
S11368602000C0B24000305CFFF71EFF0090684675
S11368704078002801D000980AE0641CDDE7280075
S11368806946087028006946487068468570009813
S113689019B0F0BD18C2000010B55B4C0320206194
S11368A060615A48A0615A49E1618021C9002162AE
S11368B00021A1626162E162206656486066102090
S11368C0A0662167E166616753A1E01D01F010F93C
S11368D05249200001F00CF92020A07110BDF1B53F
S11368E086B00C001500002001900698C768069831
S11368F0006900900098874203D20098C01B401E94
S113690005E006988068C01B00994018401E06994F
S11369108968C91B884202D306988068C01BA842B4
S113692001D2060000E02E0006984068C0190390CA
S11369300596049403980290059A04990298FEF728
S1136940CBFB0298019880190190A419AD1BBF19C3
S113695006988068874201D1002007000698C76026
S1136960002DC4D1019807B0F0BDF8B588B004007B
S11369700D001600E0680390A0680399401A029085
S1136980029886420FD260680399401800900596D9
S11369900495009F059A04993800FEF79DFB03981F
S11369A08019E06020E00298019060680399401823
S11369B00090019807900695009F079A0699380061
S11369C0FEF78AFB0298301A0190606800900198E3
S11369D00590029828180490009F059A049938009D
S11369E0FEF77AFB0198E06009B0F0BD00B5010044
S11369F00A69CB68934204D38868401EC01A801881
S1136A0001E0D01A401E00BDB0500020E8C40000D0
S1136A10585100205855002052545400F4C400002A
S1136A20F1B582B00F00150001972748029918228A
S1136A3051434018060018367069002803D0022814
S1136A4021D010D326E03000FFF7D0FF009000984B
S1136A50A84201D2002405E02C002A00019930004C
S1136A60FFF783FF17E03000FFF7C0FF00900098A6
S1136A70A84201D2009C00E02C00220001993000C1
S1136A80FFF773FF07E02A0001993000FFF727FFA3
S1136A90040000E000242000FEBDF1B50F00160044
S1136AA0094D2878002801D1FFF7F6FEEFF3108492
S1136AB0012080F31088320039000098FFF7B0FFFE
S1136AC084F31088F2BD0000B050002080B5FFF7B9
S1136AD0E3FE01BD70B504000E00A56861682800DE
S1136AE0401C814207D3206846552800401CA06002
S1136AF0E068401CE060A068616888420DD1A2682B
S1136B0021682069FFF7C9FFA168884203D00020EB
S1136B10C043E06001E00020A06070BDF7B584B020
S1136B201F000C9D059802900124012602980699E5
S1136B30884206D302980699FCF7D7F80290761C8F
S1136B40F4E7BE4200D23E000D98C0071BD4002DCE
S1136B5019D00D98800705D5002F03D13020694640
S1136B60087002E0202069460870002D0BD0AE4268
S1136B7009D26D1E684601780498FFF7ABFF0498AC
S1136B80C0680028F1D50498C06800283CD4022FBE
S1136B9001D37F1E08E005982100FCF7A6F80190B8
S1136BA001980699884202D306984443EFE7059872
S1136BB02100FCF79AF80190059801996143401A65
S1136BC0059012480199415C0498FFF783FF0498EB
S1136BD0C068002806D420000699FCF786F8040053
S1136BE0002CE4D10D98C0070ED5002D0CD0002D3B
S1136BF00AD0AE4208D26D1E20210498FFF76AFF26
S1136C000498C0680028F2D507B0F0BDD8C40000CD
S1136C10FEB582B007000A9C0298002802D50298AB
S1136C20454200E0029D01260398854206DB2800C8
S1136C300399FCF757F80500761CF5E7049886429B
S1136C4001D204980600002C06D00298002802D431
S1136C500B98400700D5641E0B98800702D5049852
S1136C60002810D00B98C0070DD4002C0BD0002C9A
S1136C7009D0A64207D2641E20213800FFF72AFF5C
S1136C80F8680028F3D5F868002836D4029800285C
S1136C9007D50298414202912D213800FFF71AFFCF
S1136CA006E00B98400703D52B213800FFF712FFAD
S1136CB0F868002821D40B988007800F022810D18F
S1136CC0049800280DD1002C0BD0002C09D0A6422A
S1136CD007D2641E30213800FFF7FCFEF868002854
S1136CE0F3D5F868002808D40B9801900094049B0D
S1136CF0039A02993800FFF711FF05B0F0BDF5B50E
S1136D009BB00C000AA80590402006900020079034
S1136D101B9809900020089020780700641C380014
S1136D20C0B2002800D11BE13800C0B2252800D031
S1136D300DE10020050001210291227817003A009C
S1136D40D2B2232A13D02B2A0CD02D2A02D0302AD7
S1136D5003D011E00D43641C0FE02A000225154303
S1136D60641C0AE02A0004251543641C05E02A007B
S1136D7008251543641C00E00290029A002ADCD125
S1136D80039021780F003900C9B2302903DB3900A0
S1136D90C9B23A2906DB049020780100C9B22E2931
S1136DA020D109E0641C03990A2251433A00D2B26B
S1136DB0891830390391E4E7641C21780800010044
S1136DC0C9B2302903DB0100C9B23A2900DB09E06A
S1136DD0641C04990A2251430200D2B28918303942
S1136DE00491EAE727783800C0B26C2803D0380051
S1136DF0C0B2682803D1641C20780700F3E7380088
S1136E00C0B2252800D19BE058284ED063280AD070
S1136E1064281CD070287BD073285DD075282DD0B1
S1136E20782842D091E01C9800681C9908601C984E
S1136E30006800681C990968091D1C9A1160029079
S1136E40029E3100C9B205A8FFF744FE7DE01C98FC
S1136E5000681C9908601C98006800681C990968FF
S1136E60091D1C9A11600290019503980090049BDF
S1136E700A22029905A8FFF7CBFE66E01C98006879
S1136E801C9908601C98006800681C990968091D11
S1136E901C9A11600290019503980090049B0A22A9
S1136EA0029905A8FFF73AFE4FE01C9800681C9968
S1136EB008601C98006800681C990968091D1C9AE0
S1136EC011600290019503980090049B102202998E
S1136ED005A8FFF723FE38E01C9800681C99086099
S1136EE01C98006806681C980068001D1C990860BE
S1136EF030780700761C3800C0B2002807D039006B
S1136F00C9B205A8FFF7E6FD08980028F0D51CE0F3
S1136F101C9800681C9908601C98006800681C99FB
S1136F200968091D1C9A1160029000200190082034
S1136F30009008231022029905A8FFF7EFFD04E052
S1136F40252105A8FFF7C6FDFFE7641C04E039000E
S1136F50C9B205A8FFF7BEFD0898002800D4DBE6F7
S1136F60089801280BDB0798002804D0079A0AA97F
S1136F701B98FFF792FD0898079940180890089805
S1136F801DB0F0BD0CB438B505000C0004A8009089
S1136F906A4621002800FFF7B2FE01B0029930BC16
S1136FA003B00847F0B58BB004003548059006904F
S1136FB000200790089009900A90324D324F334ECA
S1136FC005A8039002960197314800902B00314A9E
S1136FD0314920000830FBF7DDFD2A002F4920004D
S1136FE0603000F0BFFD02206946087404A80390D5
S1136FF02B48029001960095264B3A00294920001F
S11370008030FBF7EAFF284A28492000C830FFF700
S113701003F9274A27492000D030FFF7FDF8264A14
S113702026492000D830FFF7F7F8254A25492000E3
S1137030E030FFF7F1F8244A24492000E830FFF754
S1137040EBF80095124B320021492000F03000F09B
S1137050BFFE104B3A00104988204000201800F071
S1137060C9FE1C49B22040002018FDF785FD1A49CD
S1137070C0204000201800F031F80BB0F0BD00BF74
S113708000127A0000E0064000F8064000E80640DE
S113709000E4064000F0064000F007400000024013
S11370A000F005400080034000500340000006400B
S11370B0405003400010064080500340002006402A
S11370C0C0500340003006400051034000400640D9
S11370D000D0074000C0024000A007400160704794
S11370E010B502680121126852090A401300DBB28C
S11370F0012B19D10D4B0468636003681B6880245D
S1137100A343046823600A4B0468A36003681B68F4
S1137110DB0A0B40DBB2002BF8D103681B685B0A67
S11371200B40DBB2002BF8D010BD000020C528D9DD
S1137130FFFF000038B505000C002100280000F016
S113714024FC0548A8600548E8600F2068600448EE
S113715028610620A88231BDF8C0000040C30000A9
S11371605C080020F3B581B01400C0252600F6B2F7
S1137170281D0090029F320000993800FDF7ACFFF3
S1137180F7BD43780B707047F3B581B01400C02588
S11371902600F6B2280028300090029F32000099A1
S11371A03800FDF799FFF7BDF5B583B00C00C02595
S11371B00C2002902800183001902600029A0199B0
S11371C03000FDF789FF082628000C3000902700C6
S11371D00C37320000993800FDF77EFF2020E07262
S11371E005B0F0BDF3B581B01400C0252600F6B299
S11371F00095029F320000993800FDF76DFFF7BD3E
S113720030B500231C001500E4B2EDB2AC4205D247
S113721020241D00EDB24C555B1CF3E730BD00008B
S113722008B4024B9C4608BC6047C0464D0200208F
S113723008B4024B9C4608BC6047C0464D0400207D
S113724038B50124724D0C21280000F0DBFD002824
S113725013D10121280000F0D5FD01280AD1A3484B
S11372600168A34A914202D00020040007E00021F3
S1137270016004E00020040001E00020040020007C
S1137280C0B232BD802000017047F0B50400200078
S113729000252E00954209D2964E4F5D4740FFB21D
S11372A0BF00F659000A70406D1CF3E71E00F6B2E9
S11372B0012E02D10026F643301AF0BDFEB5002798
S11372C001970097FFF7B0F88B48FBF710FF852470
S11372D024018A4D3A0021002800FDF70BFF80208D
S11372E040020568864806688648066086490D603F
S11372F00A6882F30988096881F3088880214902B1
S1137300BE4A116000688047F7BD70B585252D0120
S113731000247A4E220029003000FDF7EBFEFFF72F
S113732083F823213A4800F02DFE70BD80B500207B
S1137330009003230622C0210120FFF7D1F901BDEB
S1137340E0B56846762101706C4B3421595C41707C
S11373500222694658689B68984707BD80B567480C
S1137360417C002916D184210901415C012903D003
S1137370B249415C01290AD10021A14A815001216D
S1137380AE4A8154022141744068417002E00420F5
S113739000F082F901BDF8B5584C607C002802D099
S11373A0607C012832D1E06900282FD0206AE1698D
S11373B088422BD200252E006769C048205C032830
S11373C014D0FFF731F801216069FFF729FF0600A7
S11373D03000C0B2002807D1E169491E8020C000F6
S11373E03818FFF71DFF0600FFF710F83000C0B291
S11373F0002805D102206074E561A561256205E0DD
S1137400E561A5612562032000F046F9F1BD0000A5
S11374102C320020F8B59F480078012864D1374CFD
S1137420607C002802D0607C01285DD1B048205CDB
S1137430012859D1E06AA16A884255D20026370052
S11374409E48205C03282BD0300069460870300029
S113745069464870022069460870FEF7E5FF35006A
S1137460280069460978C0B2884217D28022D20027
S11374702800C0B28002201801003531606AE36A36
S1137480C0182B00DBB29B02C018FFF7D1FE070027
S11374903800C0B2002801D16D1CE1E7FEF7B6FF49
S11374A03800C0B2002813D1E06A802109014018D5
S11374B0E062E06AA16A884205D330008D496054D5
S11374C00220607401E001206074FFF739FF07E0D7
S11374D0300088496054A662E662032000F0DCF8BC
S11374E03000834960542663F1BD0000F06300203E
S11374F055AAAA55049A00009C310020C0280020F7
S1137500040001001431002010310020F8B5A34C10
S1137510607C002802D0607C01286DD126001136E1
S113752001253570654820180178012902D00178B9
S1137530002957D18D4801F009F900284AD18C4817
S113754001F004F9002845D1884800688949884237
S113755007D03A482554022030700020B7496054BF
S11375604AE08F480768824800688E4940180090B6
S11375700098A021890288420ED200988A49884244
S11375800AD30123009A802149020020C043FFF757
S11375907CFE8649605002E00020844960508348A4
S11375A02058874207D025482554022030700020F7
S11375B0A249605420E0A1482554204820180178AD
S11375C0002903D1052000F067F815E005700220BA
S11375D0307011E01948255402203070002097497A
S11375E0605409E00178022906D00078032803D109
S11375F09248255402203070F1BD000008ED00E0EF
S11376004808000080B56548417C002902D0417CCF
S1137610012912D18A4941580A290CD30749415CEE
S1137620002908D19A490020FFF7ACFCFEF7FCFEC4
S1137630FFF744FE01E00121417401BD430800004D
S11376407047FEB582B00600852000010190002538
S11376500095524C2700009A01993800FDF74AFD25
S11376602660029860600398A0600498E0604F4828
S113767025503000FEF738FAFFF7E2FD012807D164
S11376806F48255001204A496054022061684870BF
S113769005B0F0BDFD3000200021404A0B005374BA
S11376A010747C4BD15070477B48007C70477A48FB
S11376B0407C704779480078704700004408000017
S11376C010B560493A4A8A181378002B07D18423ED
S11376D01B01C85400236F4C0B5101231370022269
S11376E04A7410BD574A6E4BD0546E4BD1547047F8
S11376F03E0800003D08000038B505000C00514864
S11377008461456100210A00674BC254674A815471
S1137710802149028D420CD1A02189028C4208D1DA
S11377200121634A81548169624A8918890AC161C5
S113773017E0002D0AD1082C08D102215C4A81549B
S113774081695C4A8918890AC1610AE05A498D42F3
S113775007D15A498C4204D20321554A815402214B
S1137760C1610120FFF798FF31BD0000C000010096
S1137770F87F0300DDCCBBAA38B505000C00314806
S113778001214A4A815400210A00474BC2544562F0
S11377908462C1620220FFF77FFF31BDC028002050
S11377A0FC7F03000000FFFF0140000038080000D8
S11377B043080000F4B503000022140010000C007C
S11377C0A4B2A24208D21F4C256BAD18641935250A
S11377D09E5C6655521CF2E71A4C256B0E00B6B23D
S11377E0AD1925636D462D783426A555256B802665
S11377F03601B54204D301252E002B4FE65528004F
S1137800C0B2F2BD00200F4902004A7404220A7477
S113781002000A4BCA542A4A8850704780B5094866
S1137820017C062909DA2749027C92008A58002A39
S113783003D0007C80000858804701BD3C0800004C
S113784048080000C028002010B504001248017C3C
S1137850002902D0017C052906D10E4941180A6885
S11378602300DBB2D2180A600D4941180A78012AB4
S11378700CD100220A700B49405C012804D1FFF7A7
S113788055FDFFF742FD01E0FFF73FFD10BD00008D
S113789090C4000048080000C0280020FC300020EC
S11378A041080000420800003E0800003D080000B6
S11378B044080000FF030000F05B00200108000002
S11378C038080000A00600200021016041600A0081
S11378D00272417270470022026041600123037208
S11378E042727047407A7047FEB505000E001400DE
S11378F0082100226F463800FDF7FCFB2000C0B2CF
S1137900782805D07448295A74482818FFF7E3FFEB
S11379107920285C002814D02000C0B211280FD090
S11379202000C0B212280BD02000C0B2312807D0EA
S11379302000C0B27E2803D02000C0B27F2800D12E
S11379400AE068467F21017046708470032269460C
S113795028001830FDF70AFEF7BD10B50200002319
S11379601800180080B25468A0420CD290681C0021
S1137970A4B2E400005D0C00E4B2A04201D10120F5
S113798002E05B1CEDE7002010BD70B505000C00A3
S1137990210028001830FDF7E1FF0120687000265F
S11379A03000A8703000782168540020002188221B
S11379B01201AA1803C2083AA08D49496852E08D01
S11379C048496852208E4449685289200001281889
S11379D0FFF77AFF44482818FFF776FF3F48281836
S11379E0FFF772FF310030004049884205D2310070
S11379F02A187B23D154401CF6E770BDFEB5040061
S1137A00002630006946C880300069460871370096
S1137A10350020001830FDF7EDFF01A8801C009010
S1137A20324B22007B322100793120001830FDF7DF
S1137A305FFF6946087169460420085600283CD156
S1137A407B20205C07003900C9B22000FFF785FFC6
S1137A5000282CD03500606885422ED2A068E90049
S1137A60405C3900C9B288421FD1A068E9004018BF
S1137A708078002806D07C20205CC0B2C009782120
S1137A80605402E030007821605428007A21605468
S1137A906846C28821007B3120000400A368E80006
S1137AA0181843682000984707E06D1CD3E711229B
S1137AB03900C9B22000FFF717FF08482018FFF764
S1137AC011FF012806D101206070A6700348201818
S1137AD0FFF7FAFEF7BD00008C080000A8080000BC
S1137AE0880800008A0800009C08000002080000C2
S1137AF031B48B0707D00B780370002B20D0401CC7
S1137B00491C8B07F7D1164CE501830722D104C920
S1137B10131B93432B4205D104C004C9131B934385
S1137B202B42F9D0FF231A42027009D0120A1A42DA
S1137B30427005D0120A1A42827001D0120AC27031
S1137B4031BC70470270120A4270120A8270120A23
S1137B50C270001D04C9131B93432B42F2D0E1E70A
S1137B6001010101F8B504000F00150027606560EC
S1137B700026A660E0208002E060802040052061AD
S1137B80802000026061200000F002F92076E661A6
S1137B90207E002800D06661200000F001F8F1BDCD
S1137BA0F1B489B0012069460871099909680791FF
S1137BB0002106916A461279520002231A40069265
S1137BC0069A079B1A606A46D070099A1268059152
S1137BD06B46DB781B01102423400593059B13603F
S1137BE06B469870099B1B6804916C46A4786401E9
S1137BF020252C400494049C1C606C466070099CF5
S1137C00246803916D466D78AD0140263540039597
S1137C10039D25606D462870099D2D6802916E466E
S1137C203678F60008273E400296029E2E60099E92
S1137C30366808910100C9B28900042739403160CF
S1137C400AB0F0BC7047F0B50100002528000122FD
S1137C5013000C681E00F6B2F60180273E40266031
S1137C600B681B68DB091340DBB2002BF8D00B68F0
S1137C701B685B091340DBB2002B0CD10B681B683B
S1137C801B091340DBB2002B05D10B681B681340A2
S1137C90DBB2002B00D01000C0B2F0BDFFB587B03E
S1137CA000242700250009A80078402801DB0120D2
S1137CB007000A98002801D1012007003800C0B24B
S1137CC000284DD10798006801260068C1093000DA
S1137CD00840C0B2002802D10220070040E0079803
S1137CE0FFF75EFF08206946C870200069464870A7
S1137CF00798006805900294FF20049005996A464D
S1137D0052788918097F049A91436A46D378049A71
S1137D101A400A430292029A05996B465B78C91885
S1137D200A7709A909786A46917069460E7007991D
S1137D300E6801940390684600783018007F039918
S1137D40884369468978039A0A400243019201985C
S1137D5069460978711808770798FFF774FF0700D8
S1137D603800C0B200280FD12500082D0CD22800FD
S1137D70C01D0799096822000300DBB2CB181B7FE2
S1137D800A9E73556D1CF0E73800C0B20BB0F0BD0D
S1137D907CB50500082200216846FDF779F9002624
S1137DA03400FF20694608706B4600220021280039
S1137DB0FFF774FF01000800C0B2002805D168462F
S1137DC00078800701D4012004002000C0B276BDF1
S1137DD010B4019C016042608360C46010BC7047B1
S1137DE000B5BFF34F8F054805490860BFF34F8FB7
S1137DF000BFFDE701604260836070470400FA053C
S1137E000CED00E030B50200002318000C00E4B2D1
S1137E100D2C01DBC0B2B4E00C00E4B2002C14D091
S1137E20022C29D01CD3042C3ED031D3062C53D0A1
S1137E3046D3082C68D05BD30A2C7DD070D30C2C8D
S1137E4000D191E000D283E09AE0156801242D6806
S1137E502540EDB2012D01D1200000E018008FE093
S1137E60156801242D686D082540EDB2012D01D15E
S1137E70200000E0180083E0156801242D68AD0897
S1137E802540EDB2012D01D1200000E0180077E07B
S1137E90156801242D68ED082540EDB2012D01D1AE
S1137EA0200000E018006BE0156801242D682D09FE
S1137EB02540EDB2012D01D1200000E018005FE063
S1137EC0156801242D686D092540EDB2012D01D1FD
S1137ED0200000E0180053E0156801242D68ED0926
S1137EE02540EDB2012D01D1200000E0180047E04B
S1137EF0156801242D682D0A2540EDB2012D01D10C
S1137F00200000E018003BE0156801242D686D0A8C
S1137F102540EDB2012D01D1200000E018002FE032
S1137F20156801242D68AD0A2540EDB2012D01D15B
S1137F30200000E0180023E0156801242D68ED0AF4
S1137F402540EDB2012D01D1200000E0180017E01A
S1137F50156801242D682D0B2540EDB2012D01D1AA
S1137F60200000E018000BE0156801242D686D0B5B
S1137F702540EDB2012D01D1200000E01800FFE7FB
S1137F80C0B230BDF3B581B0304801998968802210
S1137F9088506A46127A002A5AD0022A00D187E011
S1137FA06ED3042A00D1B3E000D299E0062A00D1AE
S1137FB0DEE000D2C4E0082A00D109E100D2EFE0FB
S1137FC00A2A00D134E100D21AE10C2A00D15FE17F
S1137FD000D245E10E2A00D18AE100D270E1102AD4
S1137FE000D1B5E100D29BE1122A00D1E0E100D238
S1137FF0C6E1142A00D10BE200D2F1E1162A00D125
S113800036E200D21CE2182A00D161E200D247E233
S11380101A2A00D18CE200D272E21C2A00D1B7E203
S113802000D29DE21E2A00D1EAE200D2CCE2202A4C
S113803000D11DE300D2FFE2222A00D150E300D296
S113804032E3232A00D167E369E300BF5245535565
S113805001200100019A9268546801239C430B009B
S1138060DBB20340234353600024019DAD686E6876
S11380700127BE432700FFB23840304368604EE317
S113808001200100019A9268946801239C430B002B
S1138090DBB20340234393600024019DAD68AE68C6
S11380A00127BE432700FFB238403043A86036E3BF
S11380B001200100019A9268D46801239C430B00BB
S11380C0DBB203402343D3600024019DAD68EE6816
S11380D00127BE432700FFB238403043E8601EE367
S11380E001200100019A9268146901239C430B004A
S11380F0DBB20340234313610024019DAD682E6964
S11381000127BE432700FFB238403043286106E30D
S113811001200100019A9268546901239C430B00D9
S1138120DBB20340234353610024019DAD686E69B3
S11381300127BE432700FFB2384030436861EEE2B6
S113814001200100019A9268946901239C430B0069
S1138150DBB20340234393610024019DAD68AE6903
S11381600127BE432700FFB238403043A861D6E25E
S113817001200100019A9268D46901239C430B00F9
S1138180DBB203402343D3610024019DAD68EE6953
S11381900127BE432700FFB238403043E861BEE206
S11381A001200100019A9268146A01239C430B0088
S11381B0DBB20340234313620024019DAD682E6AA1
S11381C00127BE432700FFB2384030432862A6E2AD
S11381D001200100019A9268D46A01239C430B0098
S11381E0DBB203402343D3620024019DAD68EE6AF1
S11381F00127BE432700FFB238403043E8628EE2D5
S113820001200100019A5268146801239C430B0069
S1138210DBB20340234313600024019D6D682E6884
S11382200127BE432700FFB238403043286076E27E
S113823001200100019A5268546801239C430B00F9
S1138240DBB20340234353600024019D6D686E68D4
S11382500127BE432700FFB23840304368605EE226
S113826001200100019A5268146901239C430B0008
S1138270DBB20340234313610024019D6D682E6922
S11382800127BE432700FFB238403043286146E24D
S113829001200100019A5268546901239C430B0098
S11382A0DBB20340234353610024019D6D686E6972
S11382B00127BE432700FFB23840304368612EE2F5
S11382C001200100019A5268946901239C430B0028
S11382D0DBB20340234393610024019D6D68AE69C2
S11382E00127BE432700FFB238403043A86116E29D
S11382F001200100019A5268D46901239C430B00B8
S1138300DBB203402343D3610024019D6D68EE6911
S11383100127BE432700FFB238403043E861FEE145
S113832001200100019A5268146A01239C430B0046
S1138330DBB20340234313620024019D6D682E6A5F
S11383400127BE432700FFB2384030432862E6E1EC
S113835001200100019A5268946A01239C430B0096
S1138360DBB20340234393620024019D6D68AE6A2F
S11383700127BE432700FFB238403043A862CEE154
S113838001200100019A5268146B01239C430B00E5
S1138390DBB20340234313630024019D6D682E6BFD
S11383A00127BE432700FFB2384030432863B6E1BB
S11383B001200100019A5268546B01239C430B0075
S11383C0DBB20340234353630024019D6D686E6B4D
S11383D00127BE432700FFB23840304368639EE163
S11383E001200100019A5268146C01239C430B0084
S11383F0DBB20340234313640024019D6D682E6C9B
S11384000127BE432700FFB238403043286486E189
S113841001200100019A5268546C01239C430B0013
S1138420DBB20340234353640024019D6D686E6CEA
S11384300127BE432700FFB23840304368646EE131
S113844001200100019A5268946C01239C430B00A3
S1138450DBB20340234393640024019D6D68AE6C3A
S11384600127BE432700FFB238403043A86456E1D9
S113847001200100019A5268146D01239C430B00F2
S1138480DBB20340234313650024019D6D682E6D08
S11384900127BE432700FFB23840304328653EE140
S11384A001200100019A5268146E01239C430B00C1
S11384B0DBB20340234313660024019D6D682E6ED6
S11384C00127BE432700FFB238403043286626E127
S11384D001200100019A5268546E01239C430B0051
S11384E0DBB20340234353660024019D6D686E6E26
S11384F00127BE432700FFB23840304368660EE1CF
S113850001200100019A5268946E01239C430B00E0
S1138510DBB20340234393660024019D6D68AE6E75
S11385200127BE432700FFB238403043A866F6E077
S113853001200100019A5268D46E01239C430B0070
S1138540DBB203402343D3660024019D6D68EE6EC5
S11385500127BE432700FFB238403043E866DEE01F
S113856001200100019A5268146F01239C430B00FF
S1138570DBB20340234313670024019D6D682E6F13
S11385800127BE432700FFB2384030432867C6E0C6
S113859001200100019A52688023D45801239C438E
S11385A00B00DBB203402343802413510024019DBC
S11385B06D688026AE590127BE432700FFB23840BC
S11385C030438026A851AAE001200100019A526894
S11385D08423D45801239C430B00DBB20340234380
S11385E0842413510024019D6D688426AE5901270B
S11385F0BE432700FFB2384030438426A8518EE0A2
S113860001200100019A52689023D45801239C430D
S11386100B00DBB203402343902413510024019D3B
S11386206D689026AE590127BE432700FFB238403B
S113863030439026A85172E001200100019A52684B
S11386409C23D45801239C430B00DBB203402343F7
S11386509C2413510024019D6D689C26AE5901276A
S1138660BE432700FFB2384030439C26A85156E051
S113867001200100019A52689423D45801239C4399
S11386800B00DBB203402343942413510024019DC7
S11386906D689426AE590127BE432700FFB23840C7
S11386A030439426A8513AE001200100019A52680F
S11386B0C823D45801239C430B00DBB2034023435B
S11386C0C82413510024019D6D68C826AE590127A2
S11386D0BE432700FFB238403043C826A8511EE0ED
S11386E001200100019A5268CC23D45801239C43F1
S11386F00B00DBB203402343CC2413510024019D1F
S11387006D68CC26AE590127BE432700FFB238401E
S11387103043CC26A85102E0FFF762FBFFE70020BC
S11387200199896880228850F7BD000008B4024B83
S11387309C4608BC6047C0460100002008B4024BB8
S11387409C4608BC6047C046A7000020F0B595B021
S11387500400002528006946C8736007400F0028FC
S113876001D00120CAE067480068029002980068BE
S113877001260068C0093040C0B2002801D1092098
S1138780BCE00298FFF7D2FF68468673280069466A
S113879008710298006814900995FF2013901499A9
S11387A06A4612798918097F139A91436A46927B23
S11387B0139B13400B4309930999149A6B461B7935
S11387C0D218117721006A4651736946CE70029916
S11387D0096812910895119012996A46D2788918FD
S11387E0097F119A91436A46527B119B13400B43B4
S11387F008930899129A6B46DB78D2181177210AEC
S11388006A46117302216A469170029909681091AF
S113881007950F9010996A4692788918097F0F9AE4
S113882091436A46127B0F9B13400B4307930799AE
S1138830109A6B469B78D21811772100090C6A466E
S1138840D17103216A465170029909680E91069507
S11388500D900E996A4652788918097F0D9A9143B2
S11388606A46D2790D9B13400B43069306990E9AE0
S11388706B465B78D2181177210E6A4691710421F8
S11388806A461170029909680C9105950B900C9930
S11388906A4612788918097F0B9A91436A4692793D
S11388A00B9B13400B43059305990C9A6B461B785D
S11388B0D218117729006A465171052702990E686A
S11388C004950A903800C0B23018007F0A99884392
S11388D0694649790A9A0A40024304920498390085
S11388E0C9B2711808770298FFF728FF0100080041
S11388F0C0B2002801D10B2000E02800C0B215B09E
S1138900F0BD0000F05B0020F1B489B0012069469D
S11389100871099909680791002106916A4612793C
S1138920520002231A400692069A079B1A606A466E
S1138930D070099A126805916B46DB781B011024EC
S113894023400593059B13606B469870099B1B6835
S113895004916C46A478640120252C400494049C62
S11389601C606C466070099C246803916D466D78A8
S1138970AD01402635400395039D25606D46287062
S1138980099D2D6802916E463678F60008273E4010
S11389900296029E2E60099E366808910100C9B2B3
S11389A089000427394031600AB0F0BC7047F0B543
S11389B0010000252800012213000C681E00F6B2F5
S11389C0F60180273E4026600B681B68DB091340D4
S11389D0DBB2002BF8D00B681B685B091340DBB2D9
S11389E0002B0CD10B681B681B091340DBB2002B56
S11389F005D10B681B681A40D2B2002A01D00722A5
S1138A001000C0B2F0BDF2B584B004000025280007
S1138A106946887028006946487020680126006805
S1138A20C10A30000840C0B200280ED16846007C5C
S1138A3001280AD160680068010D30000840C0B206
S1138A40012802D130006946487020680068C109D5
S1138A5030000840C0B2002801D109206DE0200098
S1138A60FFF752FF0D20694608702900226801951E
S1138A70FF2002900B00DBB2D3181F7F029B9F43A1
S1138A80BC466B461F78029B3B4067463B430193C1
S1138A90019B0F00FFB2D7193B776B461B7C002B61
S1138AA001D0370000E02F0031006A4611702168C0
S1138AB00391019502900398694609784018007F54
S1138AC0029988433900C9B2029A0A4002430192CA
S1138AD0019803996A461278891808772000FFF7ED
S1138AE066FF6946097C002909D021680968CA0A19
S1138AF031001140C9B2002901D10521080069469D
S1138B00097C002909D1216809680A0B3100114048
S1138B10C9B2002901D1052108000100C9B2002908
S1138B200BD169464978002907D021683200D2B2B6
S1138B30520380239B011A400A60C0B205B0F0BD05
S1138B4010B50400824804602000FFF7DDFE002019
S1138B50E06110BDF3B595B0002738006946087090
S1138B607B48046815988005800D002803D00120F7
S1138B7069460870E7E038003D001698854200D346
S1138B80E1E0206801260068C10930000840C0B255
S1138B90002803D1092069460870D4E02000FFF7BB
S1138BA0B3FE05216846017338006A469071206857
S1138BB014900997FF201390149A6B469B79D2184E
S1138BC0137F139A93439C466A46137B139A1A4065
S1138BD063461A430992099B9C46149B6A46927900
S1138BE09A1863461377159A6B46DA7232006B460D
S1138BF05A712268129208971190129A6B465B7907
S1138C00D218137F119A93439C466A46D37A119AD9
S1138C101A4063461A430892089B9C46129B6A4674
S1138C2052799A1863461377159AAB02D218120A2E
S1138C306B469A7202226B461A7122681092079749
S1138C400F90109A6B461B79D218137F0F9A934397
S1138C509C466A46937A0F9A1A4063461A430792CF
S1138C60079B9C46109B6A4612799A1863461377B1
S1138C70159AAB02D218120C6B465A7203226B4639
S1138C80DA7022680E9206970D900E9A6B46DB7886
S1138C90D218137F0D9A93439C466A46537A0D9AD1
S1138CA01A4063461A430692069B9C460E9B6A46EC
S1138CB0D2789A1863461377159AAB02D218120E1B
S1138CC06B461A7204226B469A7022680C920597BE
S1138CD00B900C9A6B469B78D218137F0B9A934394
S1138CE09C466A46137A0B9A1A4063461A430592C5
S1138CF0059B9C460C9B6A4692789A1863461377A8
S1138D006A46D6716A465170266804970A90684686
S1138D1040783018007F0A9988436946C9790A9ACD
S1138D200A40024304920498694649787118087706
S1138D302000FFF73CFE694608706846007800286A
S1138D4001D16D1C19E76846007817B0F0BD00002A
S1138D50F05B0020F7B598B00025280069464874F8
S1138D60874800680190072018990140002901D024
S1138D70012501E11A990840002801D00325FBE0F0
S1138D8028006946087002950B9501980068012730
S1138D900068C10A38000840C0B2012802D1380076
S1138DA06946087068460078002803D000210198BD
S1138DB0FFF729FE18988005800D0B900B98A021D1
S1138DC0490544182E001A98864205D21998805DE8
S1138DD02070641C761CF6E7019800680068C109DD
S1138DE038000840C0B2002801D10925BCE0019830
S1138DF0FFF78AFD062069460874280069468872D0
S1138E000198006816900A95FF20159016996A46F5
S1138E10927A8918097F159A91436A46137C159AA8
S1138E201A400A430A920A9A16996B469B7AC91801
S1138E300A7718996A46D17369464F72019909688D
S1138E4014910995139014996A46527A8918097FE6
S1138E50139A91436A46D27B139B13400B430993A5
S1138E600999149A6B465B7AD21811771899090AF2
S1138E706A46917302216A46117201990968129136
S1138E800895119012996A46127A8918097F119AE5
S1138E9091436A46927B119B13400B4308930899B4
S1138EA0129A6B461B7AD21811771899090C6A46E4
S1138EB0517303216A46D17001990968109107958D
S1138EC00F9010996A46D2788918097F0F9A9143B6
S1138ED06A46527B0F9B13400B4307930799109AE2
S1138EE06B46DB78D21811771899090E6A4611730C
S1138EF004216A469170019909680E9106950D90B6
S1138F000E996A4692788918097F0D9A91436A46A8
S1138F10127B0D9B13400B43069306990E9A6B46E6
S1138F209B78D21811771A99C908491E6A46D172DA
S1138F3005216A46517001990F6805950C906846A1
S1138F4040783818007F0C9988436946C97A0C9A8E
S1138F500A400243059205986946497879180877CA
S1138F600198FFF724FD050068460078002803D027
S1138F7001210198FFF747FD2800C0B21BB0F0BDE6
S1138F80F05B002000220260416001230372427200
S1138F90704770B504000E0015009E48215A9E4883
S1138FA02018FFF7EFFF7820205C012806D02A0064
S1138FB092B2310020001830FCF7D8FA70BDFEB52B
S1138FC005000E001400082100226F463800FCF74B
S1138FD091F82000C0B2782805D08E48295A8E48CE
S1138FE02818FFF7CFFF7920285C002814D0200030
S1138FF0C0B211280FD02000C0B212280BD020001C
S1139000C0B2312807D02000C0B27E2803D020008F
S1139010C0B27F2800D10AE068467F210170467003
S113902084700322694628001830FCF79FFAF7BDC4
S113903030B5002003000421020013000C00DBB251
S1139040E4B2A34208D2754B1400E4B214256C4375
S11390501B191871521CF0E730BDFFB581B0070031
S113906000252E002C0028006946087029002A00DB
S1139070002F02D10A98058032E03878C0B2000986
S11390806B46187038780007000F6B46587028003C
S113909001006A461278C9B291420BD20100C9B2EA
S11390A0791849780322121AD200914031430E00F4
S11390B0401CEDE7280069464978C0B288420BD2CB
S11390C02800C0B2381840790321491BC9008840E0
S11390D0204304006D1CEDE721003000FEF70CFB7B
S11390E005B0F0BD7047FBB504001700089D2E883D
S11390F0FEF7DAFA012814D1FEF7D9FA0100C9B251
S1139100022908D10121320092B2B954761C0021FF
S1139110424A11710DE00221320092B2B954761C18
S113912007E00320310089B27854761C00203B49C3
S113913008712E80F7BDF8B504000F0015001E005D
S1139140FEF760FBF1BD7047FBB504001700089DF6
S11391502E88FEF7A9FA042822D1FEF7A8FA0128DE
S113916005D10220310089B27854761C18E0FEF74C
S11391709EFA022814D1FEF79DFA012808D1012095
S1139180310089B27854761C00202549087007E024
S11391900320310089B27854761C002020490870DD
S11391A02E80F7BDF8B504000F0015001E00FEF771
S11391B029FBF1BD7047FBB504001700089D2E88FC
S11391C0FEF772FA042822D1FEF771FA012805D1BC
S11391D00220310089B27854761C18E0FEF767FA51
S11391E0022814D1FEF766FA012808D101203100C3
S11391F089B27854761C00200849087607E00320D9
S1139200310089B27854761C0020044908762E80F7
S1139210F7BD00008C080000A80800000C0800201E
S113922038080020704770477047F7B5FFB087B023
S11392300026049630006946087330006946488168
S11392403400300069460870042069464873802061
S113925080000190320005AD01992800FBF74AFF18
S113926030006946088188A8008886998968869AAA
S11392707A23D25CD2008918497889B2884205D20F
S1139280132231218698FFF79AFE2BE17F278798D6
S11392904078384069460873879880780002879937
S11392A0C97840186946C88188A80088001F6946A3
S11392B0488168464089002802D08798001D0490A0
S11392C0350028006946497BC0B2884234D28748B9
S11392D02900C9B214225143415A6A46D2899142A3
S11392E028D1869949782A00D2B214235A43821885
S11392F09278914218D12900C9B2142251434118DD
S1139300C97800290FD02900C9B21422514340184A
S1139310C07886998978884205D03322312186988D
S1139320FFF74DFEDEE007E0222231218698FFF7A9
S113933046FED7E06D1CC4E728006946497BC0B2ED
S1139340884205D3312231218698FFF738FEC9E0DF
S1139350802080000190009605AC009A01992000BD
S1139360FBF7C8FE05AC71202070879840786070C8
S113937087988078A0708798C078E0700420694648
S113938008816846007B012805D000D281E00328CB
S11393905BD02CD37DE055482900C9B21422514337
S11393A040180079012808D12770312060702420EA
S11393B0A07003206946088118E04C4E02A8009072
S11393C080239B0005AA68464189049884462F009F
S11393D0FFB214204743F01987686046B84701205C
S11393E02900C9B214225143711808715AE03F4848
S11393F02900C9B2142251434018007900281BD017
S113940002A8009080239B0005AA6846418904981D
S11394100190364884462F00FFB21420474360462B
S1139420C019C7680198B84730482900C9B2142246
S113943051434018067107E02770312060702420E2
S1139440A0700320694608812CE0284E2800C0B291
S11394501421484330180079002811D002A8009044
S113946080239B0005AA684641890498B4462F00CE
S1139470FFB2142677436646F6193669B04707E00B
S11394802770312060702420A07003206946088171
S113949008E02770312060701220A0700320694614
S11394A008811FE068460089042809DB20787128B8
S11394B006D16846028905A98698FFF76AFD11E07E
S11394C068460089032808D120787F2805D1A2782E
S11394D031218698FFF773FD04E024223121869818
S11394E0FFF76DFD7FB00AB0F0BD00000C0800204E
S11394F0002202604160012303724272704770B51A
S113950004000E0015009648215A96482018FFF7CB
S1139510EFFF7820205C012806D02A0092B23100A7
S113952020001830FCF722F870BDFEB505000E00CF
S11395301400082100226F463800FBF7DBFD2000F1
S1139540C0B2782805D08648295A86482818FFF7DB
S1139550CFFF7920285C002814D02000C0B2112845
S11395600FD02000C0B212280BD02000C0B2312886
S113957007D02000C0B27E2803D02000C0B27F28CC
S113958000D10AE068467F2101704670847003228E
S1139590694628001830FBF7E9FFF7BDFAB583B038
S11395A00400150001A870490A68026088200001BF
S11395B0201803C8009001A8009901700099090AB5
S11395C041700099090CC9B2427807235A4389189B
S11395D081700099090EC9B2027803235A4389188D
S11395E0C1706846007C042819D3042001000A9A3B
S11395F011806946097BA278914208D10290002625
S11396002F00320002993800FBF774FD07E0029046
S113961001AE2F00029A31003800FBF75DFD05B062
S1139620F0BDFEB504002000C0B2012802D0092814
S113963046D093E04D4D68460E782F7877400770FA
S11396404E786F78774047708E78AF787740877020
S1139650CE78ED787540C57001ADC678F0273740F7
S11396602F70C678B700BC263E404778BF07BF0FAF
S113967037436F7046783700FFB2BF08BC4607789F
S1139680C0263E4067463E43AE7006783601807879
S11396900007000F3043E87028781E78B0420BD1E1
S11396A068785E78B04207D1A8789E78B04203D13A
S11396B0E878DD78A84201D0002050E001204EE097
S11396C02A4D68460E782F78774007704E786F7869
S11396D0774047708E78AF7877408770CE78ED7892
S11396E07540C57001AD4678B700BC468778F02652
S11396F03E4067463E432E700678F6B2B6083B27D6
S11397003740BC4647787E263E4067463E436E70EF
S1139710C6783700FFB23F09BC4607782C263E4086
S113972067463E43AE7086783601C0787D27074091
S11397303743EF7028781E78B0420BD168785E7892
S1139740B04207D1A8789E78B04203D1E878DD789A
S1139750A84201D0002002E0012000E00020FEBD6C
S11397608C080000A8080000FCC4000000C500002C
S1139770F7B586B000206946887208210020009061
S113978003AC009A2000FBF7B5FC00206946C880B2
S11397900020694608810020694648716846008CAB
S11397A006998968069A7A23D25CD2008918497886
S11397B089B2884205D2132227210698FFF7B5FE05
S11397C014E106984078012805D122222721069821
S11397D0FFF7ABFE0AE1079840784006400E694661
S11397E0087103AF6720387068460079787068465E
S11397F00079C00700D47FE0002630007C4908705F
S113980034002000C0B2022837DA7A4D6846007965
S11398102100C9B20901695C88422CD12000C0B280
S11398200001281880782100C9B209016918497813
S113983088421FD206988821090140180CC80838AC
S11398402000C0B200012818083003C8121A8B4146
S1139850694800218B4208DC01DB824205D23622B2
S113986027210698FFF761FEC0E02000C0B2000186
S11398702818467001E0641CC3E72000C0B2022827
S113988005DB312227210698FFF74FFEAEE00620C4
S11398906946088101A8801C009068460389DBB2F0
S11398A0BA1C684601790698FFF778FE6846C088B6
S11398B000281BD06846C288921C92B203A906985D
S11398C0FFF71DFE68460079494908706846C0885C
S11398D04A4908806846C088009003A8851C484E01
S11398E0009A29003000FBF7F7FB7FE031222721A3
S11398F00698FFF71AFE79E03D4D6846007929780D
S1139900491C884205D0242227210698FFF70DFE22
S11399106CE06846008C801E80B200900798831C1F
S11399203648028836492878FFF77BFE6946487135
S113993068464079012822D1022203A90698FFF73C
S1139940DEFD00200100297069460979491E069A46
S1139950917004002100C9B2022947DA25496A46F8
S113996012792300DBB21B01CB5C9A4205D10200C1
S11399702300DBB21B01C9184A70641CEAE73522D4
S113998027210698FFF7D1FD00242000C0B2022849
S11399902CDA184A28782100C9B20901515C88429E
S11399A022D12000C0B2000110184078401C2100D0
S11399B0C9B20901511848702000C0B20001101842
S11399C080782100C9B209015118497888420BD224
S11399D0069888210901401803C82300DBB21B0143
S11399E0D218083203C2083A641CCEE709B0F0BDAD
S11399F0D55500208006002010270000D0550020F7
S1139A008055002000000000963007772C610EEE90
S1139A10BA51099919C46D078FF46A7035A563E9C1
S1139A20A395649E3288DB0EA4B8DC791EE9D5E0E8
S1139A3088D9D2972B4CB609BD7CB17E072DB8E7E7
S1139A40911DBF906410B71DF220B06A4871B9F33C
S1139A50DE41BE847DD4DA1AEBE4DD6D51B5D4F475
S1139A60C785D38356986C13C0A86B647AF962FDDA
S1139A70ECC9658A4F5C0114D96C0663633D0FFA27
S1139A80F50D088DC8206E3B5E10694CE44160D52D
S1139A90727167A2D1E4033C47D4044BFD850DD217
S1139AA06BB50AA5FAA8B5356C98B242D6C9BBDB2A
S1139AB040F9BCACE36CD832755CDF45CF0DD6DC25
S1139AC0593DD1ABAC30D9263A00DE518051D7C8CC
S1139AD01661D0BFB5F4B42123C4B3569995BACF57
S1139AE00FA5BDB89EB802280888055FB2D90CC678
S1139AF024E90BB1877C6F2F114C6858AB1D61C1F1
S1139B003D2D66B69041DC760671DB01BC20D2980F
S1139B102A10D5EF8985B1711FB5B606A5E4BF9F9C
S1139B2033D4B8E8A2C9077834F9000F8EA809968F
S1139B3018980EE1BB0D6A7F2D3D6D08976C6491FA
S1139B40015C63E6F4516B6B62616C1CD830658513
S1139B504E0062F2ED95066C7BA5011BC1F40882F0
S1139B6057C40FF5C6D9B06550E9B712EAB8BE8B31
S1139B707C88B9FCDF1DDD62492DDA15F37CD38CBA
S1139B80654CD4FB5861B24DCE51B53A7400BCA3B8
S1139B90E230BBD441A5DF4AD795D83D6DC4D1A4EA
S1139BA0FBF4D6D36AE96943FCD96E34468867ADC1
S1139BB0D0B860DA732D0444E51D03335F4C0AAA60
S1139BC0C97C0DDD3C710550AA41022710100BBE63
S1139BD086200CC925B56857B3856F2009D466B9AA
S1139BE09FE461CE0EF9DE5E98C9D9292298D0B0DF
S1139BF0B4A8D7C7173DB359810DB42E3B5CBDB78C
S1139C00AD6CBAC02083B8EDB6B3BF9A0CE2B6030C
S1139C109AD2B1743947D5EAAF77D29D1526DB04C1
S1139C208316DC73120B63E3843B64943E6A6D0D0C
S1139C30A85A6A7A0BCF0EE49DFF099327AE000A57
S1139C40B19E077D44930FF0D2A3088768F2011EEA
S1139C50FEC206695D5762F7CB67658071366C1981
S1139C60E7066B6E761BD4FEE02BD3895A7ADA10A2
S1139C70CC4ADD676FDFB9F9F9EFBE8E43BEB71783
S1139C80D58EB060E8A3D6D67E93D1A1C4C2D8380D
S1139C9052F2DF4FF167BBD16757BCA6DD06B53F73
S1139CA04B36B248DA2B0DD84C1B0AAFF64A0336B2
S1139CB0607A0441C3EF60DF55DF67A8EF8E6E3131
S1139CC079BE69468CB361CB1A8366BCA0D26F257A
S1139CD036E2685295770CCC03470BBBB9160222C7
S1139CE02F260555BE3BBAC5280BBDB2925AB42BDC
S1139CF0046AB35CA7FFD7C231CFD0B58B9ED92CF1
S1139D001DAEDE5BB0C2649B26F263EC9CA36A7555
S1139D100A936D02A906099C3F360EEB856707720C
S1139D2013570005824ABF95147AB8E2AE2BB17B73
S1139D30381BB60C9B8ED2920DBED5E5B7EFDC7CFA
S1139D4021DFDB0BD4D2D38642E2D4F1F8B3DD6851
S1139D506E83DA1FCD16BE815B26B9F6E177B06F4C
S1139D607747B718E65A0888706A0FFFCA3B066639
S1139D705C0B0111FF9E658F69AE62F8D3FF6B61C6
S1139D8045CF6C1678E20AA0EED20DD75483044E68
S1139D90C2B30339612667A7F71660D04D476949F6
S1139DA0DB776E3E4A6AD1AEDC5AD6D9660BDF4009
S1139DB0F03BD83753AEBCA9C59EBBDE7FCFB247BC
S1139DC0E9FFB5301CF2BDBD8AC2BACA3093B353A1
S1139DD0A6A3B4240536D0BA9306D7CD2957DE54AA
S1139DE0BF67D9232E7A66B3B84A61C4021B685D83
S1139DF0942B6F2A37BE0BB4A18E0CC31BDF055AFC
S1139E008DEF022DF0B590B0012001006A469170EB
S1139E10DA4A04920499C96A0423DB4319406C4664
S1139E20A478A40004252C400C430B940B99049CA7
S1139E30E16201006C46617003920399C96A0124CE
S1139E40A1436C46647804400C430A940A99039C29
S1139E50E16200210C006D462C700292029AD26AD3
S1139E6013406A4612789200042422401A4309924D
S1139E70099A029BDA62CB4A0892CB4A0792089B62
S1139E80079C23660300C94C0194019C24680F2598
S1139E90AC431D00EDB22D072D0F25430695069CFE
S1139EA0019D2C60C24CC34D0595059D8026AC5187
S1139EB0C14D2D682D0EAD07AD0FEDB2022D2AD187
S1139EC00B006C462370BD4B5D68BD4C2C406D4649
S1139ED02D782D02F02636012E4026430296029C50
S1139EE05C600C00B44D0195019E3668B54F374057
S1139EF0BC462600F6B23704C026B6023E4067468A
S1139F003E43019F3E602B001B681B0E9B079B0F6B
S1139F10DBB2002BF7D103000092009CE4680C250F
S1139F20AC431D00EDB2AD000C262E402643019635
S1139F30019C009DEC6004001500EE680127BE43FF
S1139F402700FFB207403743EF6013001B6A9C08E9
S1139F5003002340DBB2002BF7D00B006C46637187
S1139F600892089B5B690124A3436C46647904400E
S1139F701C430F940F9B089C63610B006C46237178
S1139F800792079B9B691024A3436C462479240100
S1139F9010252C401C430E940E9B079CA3610B00C0
S1139FA06C46E3700692069B5C69874B23406C46C3
S1139FB0E4782402C025AD0025401D430D950D9B7A
S1139FC0069C636150236C46A3700592059B5B69F4
S1139FD0FE24A3436C46A4786400FE2525401D435B
S1139FE00C950C9B059C63610B006C46637004929A
S1139FF0049B5C69754B23406C466478A4028025FD
S113A000ED002C401C430B940B9B049C63610423C4
S113A0101C006D462C700392039C65696C4C2C40AB
S113A0206D462D78ED02E026B6012E4026430A96B1
S113A0300A9C039D6C6104000292029D6D690126D5
S113A040B5432600F6B206402E430996099D029EAA
S113A0507561FA256D015F4E35605F4D29605F4E75
S113A06005273760346880277F02BC42FAD3336007
S113A070584B1960296013001C6A03002340DBB2AB
S113A080002BF8D002246B461C71554B0693069D99
S113A090C826AE594B4D35406E4636793704C02636
S113A0A0B6023E402E430896089D069EC827F551E9
S113A0B009256E46F5700593059DC826AD59404E99
S113A0C02E400296029D6E46F6783702F02636013F
S113A0D03E402E430296029D059EC827F551050079
S113A0E06E46B5700493049BC8255B591025AB4399
S113A0F06D46AD782D01102635401D430795079B0D
S113A100049DC826AB516B4658702C4D6B682C4887
S113A11018406B465B781E02F0231B013340034357
S113A1206B606846047024480390039C2668254CA1
S113A13034406E4636783704C026B6023E40264385
S113A140039C266003001B681B0E9B079B0FDBB25E
S113A150022BF7D10B00154C0094009C24680F25AA
S113A160AC431D00EDB22D072D0F25430295029C33
S113A170009D2C600C000568114E01E000F00540C4
S113A1802E402500EDB22F02F0252D013D40354330
S113A19005600191019E1666064E8027F15110B0AC
S113A1A0F0BD00BF2020961900E0064000E4064000
S113A1B05245535500F0064000E8064000000240B6
S113A1C0FFF0FFFFFFFFFCFFFFFCFFFFFFFBFFFFB4
S113A1D0FFC7FFFF14E000E018E000E010E000E03B
S113A1E000F80640002202604160012303724272BB
S113A1F0704770B504000E001500B848215AB848DD
S113A2002018FFF7EFFF7820205C012806D02A00F1
S113A21092B2310020001830FBF7A8F970BDFEB5EA
S113A22005000E001400082100226F463800FAF7DA
S113A23061FF2000C0B2782805D0A848295AA84850
S113A2402818FFF7CFFF7920285C002814D02000BD
S113A250C0B211280FD02000C0B212280BD02000A9
S113A260C0B2312807D02000C0B27E2803D020001D
S113A270C0B27F2800D10AE068467F210170467091
S113A28084700322694628001830FBF76FF9F7BD84
S113A290F7B5FFB085B0050000206946488000206E
S113A2A06946C88000260020694688800024002072
S113A2B069460870802189000020029004AF029A48
S113A2C03800FAF717FF86A80088A9687A22AA5CE2
S113A2D0D2008918497889B2884205D213222221F2
S113A2E02800FFF79CFFF6E086A80088401EC00700
S113A2F005D5132222212800FFF791FFEBE086A861
S113A300008840086946488068464088002805D18E
S113A310132222212800FFF782FFDCE0622004A937
S113A320320092B28854761C0127380086A9098825
S113A33080B2884200D3BEE08598390089B2405C7F
S113A340000285993A0092B289184978084369460F
S113A350C880002001006A46117004002000A98A08
S113A36080B2884200D3A0E02869210089B2142277
S113A3704A43805A6946C988884200D093E0A87845
S113A3802969220092B214235343C91809798842D7
S113A39005D0332222212800FFF741FF9BE0300043
S113A3A080B22969220092B214235343C9188989BF
S113A3B04018801C4B49884205DB142222212800C6
S113A3C0FFF72DFF87E02869210089B214224A4350
S113A3D080188078052809D068782969220092B20B
S113A3E014235343C918C978884205D22222222152
S113A3F02800FFF714FF6EE02869210089B21422B7
S113A4004A4380188289D2B22869210089B2142370
S113A4104B43C0188168280005002B699C46230023
S113A4209BB21420584363461818036928009847C0
S113A43001206946087004A885993A0092B2895CA3
S113A440320092B28154761C85993A0092B28918EE
S113A4504978320092B28154761C68468680286915
S113A460210089B214224A43801880890390286904
S113A470210089B214224A4380188068029004A8FB
S113A480694689884618039A02993000FAF724FE2F
S113A490684680882969220092B214235343C9185C
S113A4A08989461801E0641C58E76846007800284A
S113A4B001D0BF1C39E768460078002806D0320076
S113A4C092B204A92800FFF794FE04E0312222216D
S113A4D02800FFF7A4FE7FB008B0F0BD8C08000090
S113A4E0A80800000102000000220260416001236C
S113A4F003724272704770B504000E0015009D4847
S113A500215A9D482018FFF7EFFF7820205C01288E
S113A51006D02A0092B2310020001830FBF726F84A
S113A52070BDFEB505000E001400082100226F4620
S113A5303800FAF7DFFD2000C0B2782805D08D4836
S113A540295A8D482818FFF7CFFF7920285C002866
S113A55014D02000C0B211280FD02000C0B212289D
S113A5600BD02000C0B2312807D02000C0B27E2812
S113A57003D02000C0B27F2800D10AE068467F21C2
S113A5800170467084700322694628001830FAF777
S113A590EDFFF7BD7047704770477047F4B5FFB0E3
S113A5A085B005000E000027380069464880380051
S113A5B06946087038006946087102206946487087
S113A5C0802189003A0004AC2000FAF793FD84A8A6
S113A5D00088A9687A22AA5CD2008918497889B2CD
S113A5E0884205D213222F212800FFF79AFFBDE0ED
S113A5F06878012805D122222F212800FFF791FF36
S113A600B4E070780002B178401869464880F07868
S113A610694608703C00200069464978C0B2884207
S113A62023D256482100C9B214225143415A6A46E2
S113A6305288914217D12100C9B2142251434118C2
S113A640897800290ED02100C9B214225143401840
S113A6508078A978884205D033222F212800FFF77B
S113A66060FF83E001E0641CD5E720006946497877
S113A670C0B2884205D331222F212800FFF751FFB1
S113A68074E004A86F21017071784170B178817011
S113A690F178C17068460078002802D003281CD0E5
S113A6A05FE036482100C9B2142251434118CF72E9
S113A6B02100C9B2142251434118096900290BD061
S113A6C02100C9B214225143401800698047042272
S113A6D004A92800FFF70FFF48E0284F84A800884A
S113A6E02100C9B2142251437918097A091D8842FC
S113A6F005DA22222F212800FFF713FF36E001207C
S113A7002100C9B2142251437918C8722000C0B282
S113A710142148433818007A0390301D0290200019
S113A720C0B214214843381840680190039A029932
S113A7300198FAF7D1FC01982000C0B214214843D3
S113A7403818C06800280BD02000C0B21421484338
S113A7503818C0688047042204A92800FFF7CBFEFC
S113A76004E031222F212800FFF7DBFE7FB006B082
S113A770F0BD00008C080000A8080000E4070020D9
S113A780002202604160012303724272704770B577
S113A79004000E0015002548215A25482018FFF70B
S113A7A0EFFF7820205C012806D02A0092B2310005
S113A7B020001830FAF7DAFE70BDFEB505000E0071
S113A7C01400082100226F463800FAF793FC200099
S113A7D0C0B2782805D01548295A15482818FFF71B
S113A7E0CFFF7920285C002814D02000C0B21128A3
S113A7F00FD02000C0B212280BD02000C0B23128E4
S113A80007D02000C0B27E2803D02000C0B27F2829
S113A81000D10AE068467F210170467084700322EB
S113A820694628001830FAF7A1FEF7BD8C0800002D
S113A830A808000010B50024FCF724FD801C10BDFE
S113A84010B501000020030001221300DBB2052B28
S113A8500CDA04239B1ADB000C00DC40002C03D030
S113A86005239B1A180001E0521CEEE7C0B210BD8C
S113A870F7B586B00020050001006A461170040097
S113A880070001006A465170029001006A46D170C7
S113A890060006994978012905D122223421069817
S113A8A0FFF78BFFA4E069460B8C06998A689446EF
S113A8B0069A7A21515CC90062465118497889B2D6
S113A8C08B4205D2132234210698FFF776FF8FE0DE
S113A8D0079989780907090F6A46117007998978D9
S113A8E0C9B209096A4691706946097800290BD0F2
S113A8F069460978052907D269468978002903D071
S113A90069468978052905D3312234210698FFF751
S113A91054FF6DE001000A006B461B78D2B29A42E4
S113A92008D22A02079B0D00EDB25B19DB78D5181B
S113A930491CF0E70700380069468978C0B28842AC
S113A9400BD2210207986A4612783B00DBB2D21878
S113A9508018C0780C187F1CEDE7002C05D122224A
S113A96034210698FFF729FF42E000F083F828001D
S113A97000F08EF8200000F08EF8012000F091F82D
S113A980FFF758FF02900298FFF75AFF6946487094
S113A99003A87421320092B28154761C6946497826
S113A9A00901320092B28154761C69468E800126D8
S113A9B0694649783200D2B291420FD302996A466D
S113A9C05278921BD200D1406A46928881546946DB
S113A9D08988491C6A469180761CE9E72100280091
S113A9E0FCF7CAFE6846828803A90698FFF7CFFEE3
S113A9F009B0F0BD0022026041600123037242727B
S113AA007047FEB505000E001400082100226F46B1
S113AA103800FAF76FFB2000C0B2782805D06348ED
S113AA20295A63482818FFF7E5FF7920285C002895
S113AA3014D02000C0B211280FD02000C0B21228B8
S113AA400BD02000C0B2312807D02000C0B27E282D
S113AA5003D02000C0B27F2800D10AE068467F21DD
S113AA600170467084700322694628001830FAF792
S113AA707DFDF7BD002001004E4A117001004E4AD1
S113AA8011704E4908604E4908604E49086070478D
S113AA904B49086070474B49086070474948006853
S113AAA070474949087070474748007870474348E1
S113AAB000687047F6B583B005000A2100226C4691
S113AAC02000FAF717FB6878012805D122223621E5
S113AAD02800FFF796FF66E06846008AA9687A2294
S113AAE0AA5CD2008918497889B2884205D2132217
S113AAF036212800FFF785FF55E033480078012808
S113AB0002D0022844D049E02A4C039840782070AF
S113AB10294E2078317888420BD020783178491C2E
S113AB20C9B2884205D0732236212800FFF769FF95
S113AB3039E0224F2348006839686A46128A891826
S113AB40891E884205D2712236212800FFF759FF59
S113AB5029E020783178491CC9B2884217D122787B
S113AB606846018A891E89B20398801CFCF722FE7C
S113AB70012805D138686946098A4018801E386062
S113AB8020783070684676210170217841700AE09F
S113AB90312236212800FFF734FF04E02422362135
S113ABA02800FFF72EFF05B0F0BD00008C08000060
S113ABB0A8080000D8550020D9550020945500203D
S113ABC08C55002090550020D755002091490870DD
S113ABD0704730B5010089B2142928DA00218E4A61
S113ABE00B000400A4B20C2565435419237103001F
S113ABF09BB20C245C4313191B1D1C7810252543A0
S113AC001D7003009BB20C245C4313191B1D1C789C
S113AC10402525431D7003009BB20C245C4313198B
S113AC20D98003009BB20C245C431219117230BD0D
S113AC3070B5010000231C001A0018001C00A4B207
S113AC40142C10DA744C1D00ADB20C266E43A419FA
S113AC5024796406640E22001400E4B20C4200D08D
S113AC60401C5B1CEAE780B270BDF2B50100002411
S113AC702500230020002500ADB2142D39DA664DDD
S113AC802600B6B20C277743EE19367933001E003E
S113AC90F6B216422BD06E4636880700BFB23F1D6F
S113ACA0BE4223DB2600B6B20C277743EE59360C9E
S113ACB00700BFB2CE55401C2600B6B20C2777431E
S113ACC0EE59360A0700BFB2CE55401C2600B6B274
S113ACD00C277743ED590600B6B28D55401C5D062E
S113ACE06D0E0600B6B28D55401C00E001E0641CF8
S113ACF0C1E780B2F2BDF0B50200002425002300B4
S113AD0020002500ADB2142D33DA434D2600B6B22F
S113AD100C277743EE19367933000E00B6B20700DC
S113AD20BFB23F1DBE4224DB2600B6B20C277743D8
S113AD30EE59360C0700BFB2D655401C2600B6B2F9
S113AD400C277743EE59360A0700BFB2D655401C8C
S113AD502600B6B20C277743ED590600B6B29555D6
S113AD60401C5D066D0E0600B6B29555401C641C71
S113AD70C7E780B2F0BD38B504000020050021000B
S113AD80264A891A04D09D3918D02F3935D03FE08E
S113AD900500280080B214280FDA1F48290089B260
S113ADA00C224A43805880214903884203D2280058
S113ADB080B2FFF70EFF6D1CEBE729E005002800C9
S113ADC080B2142818DA1448290089B20C224A43A4
S113ADD081588022D20391420CD3290089B20C22DB
S113ADE04A43805880210904884203D2280080B253
S113ADF0FFF7EFFE6D1CE2E70AE00500280080B2D1
S113AE00142805DA280080B2FFF7E3FE6D1CF5E78D
S113AE1031BD0000D4550020F406002033FFFF00AC
S113AE200100050000000000000000000000000018
S113AE300900050000000000000000000000000000
S113AE405D730000977300001574000041760000E4
S113AE500D750000057600000100000031070000B8
S113AE60DF070000B1070000AC3200200002000040
S113AE70AC3400202008000000000000F55D000054
S113AE80AD5C00003200F4018813000001020304E9
S113AE90050607081A6204005000000000000000C4
S113AEA01B63040050000000000000001603F000C3
S113AEB050000000000000001703F00050000000E4
S113AEC0000000008873C000500000000000000073
S113AED00100C10050000000000000000101C10099
S113AEE050000000000000000121C10050000000DB
S113AEF0000000000127C100500000000000000015
S113AF000128C10050000000000000000129C10018
S113AF1050000000000000000131C100500000009A
S113AF20000000000041C1005000000000000000CB
S113AF300151C10050000000000000000063C10086
S113AF4050000000000000000069C1005000000033
S113AF50000000000181C10050000000000000005A
S113AF600136C20050000000000000000064C1006F
S113AF7050000000000000000067C1005000000005
S113AF800000000092F0000088550020020000003C
S113AF9095A5000097A5000020F000008A55002028
S113AFA00200000099A500009BA5000001FD020914
S113AFB0000000005B900000E5900000E7900000B6
S113AFC002FD020900000000A5910000B5910000F7
S113AFD0B791000003FD0209000000003791000052
S113AFE0479100004991000004FD0209000000009F
S113AFF025920000279200002992000086F10601A4
S113B000000000009855002001000000837100003A
S113B01087F1060100000000995500200800000097
S113B0208971000080F1060100000000A155002094
S113B030080000006571000091F1060100000000A5
S113B040A955002018000000A971000093F1060121
S113B05000000000C155002004000000E57100005C
S113B06095F1060100000000C5550020080000000D
S113B07001720000002202604160012303724272E7
S113B080704770B504000E0015007E48215A7E48B2
S113B0902018FFF7EFFF7820205C012806D02A0053
S113B0A092B2310020001830FAF760FA70BDFEB594
S113B0B005000E001400082100226F463800FAF73C
S113B0C019F82000C0B2782805D06E48295A6E4875
S113B0D02818FFF7CFFF7920285C002814D020001F
S113B0E0C0B211280FD02000C0B212280BD020000B
S113B0F0C0B2312807D02000C0B27E2803D020007F
S113B100C0B27F2800D10AE068467F2101704670F2
S113B11084700322694628001830FAF727FAF7BD2D
S113B120F6B583B004000E00082100273A0001ADF3
S113B1302800F9F7DFFF3800694648706846008A3E
S113B140A1687A22A25CD2008918497889B288421F
S113B15005D2132228212000FFF7A9FF8EE0607892
S113B160012805D1222228212000FFF7A0FF85E035
S113B17070784006400E69460870B57801A86821C9
S113B180017069460978417068460078002805D046
S113B190022838D01CD3032850D06AE02800C0B25B
S113B1A0012807D02800C0B2022803D02800C0B26A
S113B1B0032807D135480770022201A92000FFF7B0
S113B1C060FF04E0312228212000FFF770FF55E0E2
S113B1D02800C0B2012807D02800C0B2022803D03A
S113B1E02800C0B2032808D101202849087002228F
S113B1F001A92000FFF745FF04E0312228212000A7
S113B200FFF755FF3AE02800C0B2012807D0280014
S113B210C0B2022803D02800C0B2032808D10220FB
S113B2201A490870022201A92000FFF72AFF04E04E
S113B230312228212000FFF73AFF1FE02800C0B286
S113B240012807D02800C0B2022803D02800C0B2C9
S113B250032808D103200D490870022201A9200007
S113B260FFF70FFF04E0312228212000FFF71FFF22
S113B27004E0122228212000FFF719FF05B0F0BDD9
S113B280000000008C080000A8080000D65500202B
S113B290002202604160012303724272704770B55C
S113B2A004000E0015002548215A25482018FFF7F0
S113B2B0EFFF7820205C012806D02A0092B23100EA
S113B2C020001830FAF752F970BDFEB505000E00E3
S113B2D01400082100226F463800F9F70BFF200004
S113B2E0C0B2782805D01548295A15482818FFF700
S113B2F0CFFF7920285C002814D02000C0B2112888
S113B3000FD02000C0B212280BD02000C0B23128C8
S113B31007D02000C0B27E2803D02000C0B27F280E
S113B32000D10AE068467F210170467084700322D0
S113B330694628001830FAF719F9F7BD8C0800009F
S113B340A8080000F6B585B005000E000024200012
S113B350694608802000694648800821220003AF1E
S113B3603800F9F7C7FE6846008BA9687A22AA5C00
S113B370D2008918497889B2884205D213222E2135
S113B3802800FFF7A2FF82E070780002B17808433A
S113B3906946088003A86E21017071784170B17804
S113B3A081702000A98A80B288426BD2286921006A
S113B3B089B214224A43805A6946098888425FD177
S113B3C02869210089B214224A4380180079002890
S113B3D00FD0A8782969220092B214235343C918C4
S113B3E00979884205D0332222212800FFF76DFF16
S113B3F04DE06846008BC01E2969220092B21423D6
S113B4005343C9188989884205D013222E21280064
S113B410FFF75BFF3BE02869210089B214224A430D
S113B42080188078032809D068782969220092B2AC
S113B43014235343C918C978884205D222222E21E5
S113B4402800FFF742FF22E02869210089B2142274
S113B4504A43801880890290F01C019028692100D9
S113B46089B214224A4380188768029A01993800E5
S113B470F9F732FE032203A92800FFF710FF06E0C4
S113B480641C8EE731222E212800FFF71EFF07B02F
S113B490F0BD000000220260416001230372427289
S113B4A0704770B504000E0015002548215A254840
S113B4B02018FFF7EFFF7820205C012806D02A002F
S113B4C092B2310020001830FAF750F870BDFEB582
S113B4D005000E001400082100226F463800F9F719
S113B4E009FE2000C0B2782805D01548295A15480D
S113B4F02818FFF7CFFF7920285C002814D02000FB
S113B500C0B211280FD02000C0B212280BD02000E6
S113B510C0B2312807D02000C0B27E2803D020005A
S113B520C0B27F2800D10AE068467F2101704670CE
S113B53084700322694628001830FAF717F8F7BD1B
S113B5408C080000A8080000F6B5FFB082B0070020
S113B5500022100069464870100069460870100007
S113B5606946488015008021890001AC2000F9F764
S113B570C1FD82A80088B9687A22BA5CD200891811
S113B580497889B2884205D2132219213800FFF77D
S113B5909EFF75E07F268198407830406946487068
S113B5A001AC592020706846407860706846407845
S113B5B0012804D0022827D00A2844D05BE082A8BE
S113B5C00088032805D0132219213800FFF77FFFD4
S113B5D056E0819880786946087068460078FFF7DD
S113B5E027FB69464880A6700120E07068464088C1
S113B5F080B2000A2071684640886071062201A961
S113B6003800FFF74EFF3BE082A80088032805D0EE
S113B610132219213800FFF75AFF31E0819880780E
S113B62069460870A67068460278FF21FE31E01C66
S113B630FFF71BFB05002A00D21C92B201A93800B7
S113B640FFF72FFF1CE082A80088022805D01322F0
S113B65019213800FFF73BFF12E0FF21FE31E01C07
S113B660FFF749FB05002A00D21C92B201A9380059
S113B670FFF717FF04E0122219213800FFF727FF14
S113B6807FB004B0F0BD00000022026041600123DD
S113B69003724272704770B504000E0015006348CF
S113B6A0215A63482018FFF7EFFF7820205C012817
S113B6B006D02A0092B2310020001830F9F756FF64
S113B6C070BDFEB505000E001400082100226F466F
S113B6D03800F9F70FFD2000C0B2782805D0534890
S113B6E0295A53482818FFF7CFFF7920285C0028EF
S113B6F014D02000C0B211280FD02000C0B21228EC
S113B7000BD02000C0B2312807D02000C0B27E2860
S113B71003D02000C0B27F2800D10AE068467F2110
S113B7200170467084700322694628001830F9F7C6
S113B7301DFFF7BDF2B582B00500170008210024F3
S113B74022006E463000F9F7D5FC3800A9687A2249
S113B750AA5CD2008918497880B289B2884205D09F
S113B760132210212800FFF7ACFF5EE00298407816
S113B7704606760E68465021017046702D49695A76
S113B78089B2090A81702B49695AC1702A49695AD8
S113B79089B2090A01712849695A4171FDF748FCC7
S113B7A03000C0B2012806D03AD303280BD018D3F6
S113B7B0042827D034E0AC706E7006226946280055
S113B7C0FFF769FF31E0AC706E700622694628000D
S113B7D0FFF761FF1548295A15482818FFF754FF49
S113B7E023E0AC706E70062269462800FFF753FF11
S113B7F00E48295A0E482818FFF746FF0120FBF788
S113B8005FFF12E0AC706E70062269462800FFF7F5
S113B81042FF0648295A06482818FFF735FF04E076
S113B820122210212800FFF74CFFF7BD8C080000FE
S113B830A8080000880800008A080000210400000D
S113B8404D0400002D050000000000004F0500001D
S113B85045060000EF070000450800001509000038
S113B8606B0900003D0A0000930A0000610B000010
S113B870B70B0000810C0000D70C0000A10D0000E4
S113B880F70D0000C50E00001F0F0000810F00001F
S113B890B90F0000E90F000023100000571000004A
S113B8A0F1100000AD110000031300006916000040
S113B8B0000000007316000097160000C116000077
S113B8C0E51600000F170000000000001B17000021
S113B8D06F170000211800004B18000075180000B5
S113B8E09F180000C9180000F31800001D1900007B
S113B8F047190000711900009B190000C5190000C8
S113B900931A0000211C00008D1C0000911D0000F2
S113B910011E0000E11E0000231F00006F1F000035
S113B920B11F000001200000432000008F20000010
S113B930D12000001D2100005F210000B121000082
S113B940F1210000452200006B2200009522000036
S113B950BB220000E52200000B2300003523000079
S113B9605B23000085230000AB230000D5230000E7
S113B970FB23000025240000B3240000CB25000095
S113B980F12500001B2600007F2600002927000067
S113B9900000000033270000000000003D270000E5
S113B9A00000000047270000C5270000AF28000062
S113B9B02D290000172A0000512A0000AD2A00009A
S113B9C0E72A00003F2B0000672B000000220260E2
S113B9D04160012303724272704770B504000E0087
S113B9E015002548215A25482018FFF7EFFF782035
S113B9F0205C012806D02A0092B2310020001830C1
S113BA00F9F7B4FD70BDFEB505000E001400082161
S113BA1000226F463800F9F76DFB2000C0B2782889
S113BA2005D01548295A15482818FFF7CFFF792063
S113BA30285C002814D02000C0B211280FD02000A8
S113BA40C0B212280BD02000C0B2312807D0200089
S113BA50C0B27E2803D02000C0B27F2800D10AE003
S113BA6068467F210170467084700322694628006D
S113BA701830F9F77BFDF7BD8C080000A80800001A
S113BA80F2B582B0040016000022150008216F46AA
S113BA903800F9F72FFB6078012805D122223721DD
S113BAA02000FFF7B0FF40E03000A1687A22A25CDA
S113BAB0D2008918497880B289B2884205D213220B
S113BAC037212000FFF79FFF2FE0772069462A00E7
S113BAD092B288546D1C2F00FEF7E6FF012802D0B5
S113BAE0022814D019E0FEF7E2FF0500FEF7D6FFA6
S113BAF0854205D0132237212000FFF784FF11E08F
S113BB003A0092B269462000FFF767FF0AE031224B
S113BB1037212000FFF777FF04E02422372120009B
S113BB20FFF771FF0020FEF7BCFFF7BD00220260A3
S113BB304160012303724272704770B504000E0025
S113BB4015002548215A25482018FFF7EFFF7820D3
S113BB50205C012806D02A0092B23100200018305F
S113BB60F9F704FD70BDFEB505000E0014000821B0
S113BB7000226F463800F9F7BDFA2000C0B27828D9
S113BB8005D01548295A15482818FFF7CFFF792002
S113BB90285C002814D02000C0B211280FD0200047
S113BBA0C0B212280BD02000C0B2312807D0200028
S113BBB0C0B27E2803D02000C0B27F2800D10AE0A2
S113BBC068467F210170467084700322694628000C
S113BBD01830F9F7CBFCF7BD8C080000A80800006A
S113BBE0FEB504000F0016000821002201AD280054
S113BBF0F9F780FAFF253100A0687A22A25CD2000E
S113BC008018407889B280B2814205D01322112174
S113BC102000FFF7A8FF37E078784006400E694619
S113BC20087001A851210170694609784170857036
S113BC3068460078012804D021D3032815D00AD3FC
S113BC401DE0032201A92000FFF777FF0121012055
S113BC50FBF748FD18E0032201A92000FFF76DFF60
S113BC6002210120FBF73EFD0EE0032201A9200082
S113BC70FFF763FF03210120FBF734FD04E01222E8
S113BC8011212000FFF76FFFF7BD000000220260C2
S113BC904160012303724272704770B504000E00C4
S113BCA015002548215A25482018FFF7EFFF782072
S113BCB0205C012806D02A0092B2310020001830FE
S113BCC0F9F754FC70BDFEB505000E001400082100
S113BCD000226F463800F9F70DFA2000C0B2782828
S113BCE005D01548295A15482818FFF7CFFF7920A1
S113BCF0285C002814D02000C0B211280FD02000E6
S113BD00C0B212280BD02000C0B2312807D02000C6
S113BD10C0B27E2803D02000C0B27F2800D10AE040
S113BD2068467F21017046708470032269462800AA
S113BD301830F9F71BFCF7BD8C080000A8080000B8
S113BD40FEB504000E001500082100226F463800DD
S113BD50F9F7D0F92800A1687A22A25CD2008918E8
S113BD60497880B289B2884205D213228521200005
S113BD70FFF7A9FF2DE06078012805D12222852153
S113BD802000FFF7A0FF24E0707847067F0E684686
S113BD90C521017047703800C0B2012802D00228C2
S113BDA009D011E00120FEF711FF022269462000AC
S113BDB0FFF773FF0DE00020FEF708FF022269463B
S113BDC02000FFF76AFF04E0122285212000FFF71C
S113BDD07AFFF7BD002202604160012303724272C0
S113BDE0704770B504000E0015004448215A4448B9
S113BDF02018FFF7EFFF7820205C012806D02A00E6
S113BE0092B2310020001830F9F7B0FB70BDFEB5D6
S113BE1005000E001400082100226F463800F9F7CF
S113BE2069F92000C0B2782805D03448295A34482A
S113BE302818FFF7CFFF7920285C002814D02000B1
S113BE40C0B211280FD02000C0B212280BD020009D
S113BE50C0B2312807D02000C0B27E2803D0200011
S113BE60C0B27F2800D10AE068467F210170467085
S113BE7084700322694628001830F9F777FBF7BD70
S113BE80F7B504000D000022160008216F463800A3
S113BE90F9F730F968460089A1687A22A25CD200D9
S113BEA08918497889B2884205D0132214212000C8
S113BEB0FFF7ADFF20E0687800043043A978090259
S113BEC00143EE780E4354206946087030000D4952
S113BED0401A03D09D3801D02F3808D13000FEF726
S113BEE04AFF012269462000FFF77BFF04E031226C
S113BEF014212000FFF78BFFF7BD00008C08000021
S113BF00A808000033FFFF00002202604160012303
S113BF1003724272704770B504000E001500254884
S113BF20215A25482018FFF7EFFF7820205C0128CC
S113BF3006D02A0092B2310020001830F9F716FB1F
S113BF4070BDFEB505000E001400082100226F46E6
S113BF503800F9F7CFF82000C0B2782805D015488A
S113BF60295A15482818FFF7CFFF7920285C0028A4
S113BF7014D02000C0B211280FD02000C0B2122863
S113BF800BD02000C0B2312807D02000C0B27E28D8
S113BF9003D02000C0B27F2800D10AE068467F2188
S113BFA00170467084700322694628001830F9F73E
S113BFB0DDFAF7BD8C080000A8080000FEB50400F7
S113BFC00E001500082100226F463800F9F792F898
S113BFD02800A1687A22A25CD2008918497880B22C
S113BFE089B2884205D013223E212000FFF7A9FF21
S113BFF015E0707847067F0E3800C0B2002809D1DA
S113C00068467E2101704770022269462000FFF7CE
S113C01082FF04E012223E212000FFF792FFF7BDC9
S113C020F0B587B02548029025482649069126494F
S113C03001912649264A0592264A274B0493274B09
S113C0400093274B274C0394069C844207D0047822
S113C050029D2C70029C641C0294401CF4E7059C15
S113C0608C4207D00C78019D2C70019C641C0194B7
S113C070491CF4E7049C944203D000241470521C1D
S113C080F8E7039C9C4207D01C78009D2C705B1C35
S113C090009C641C0094F4E70024134DAD08AC42EA
S113C0A007D2124DA600AD59114EA700F551641CDC
S113C0B0F3E70F4D0F4E356007B0F0BD800600204A
S113C0C020AE000074B000000000002008890000C9
S113C0D0848F000000200020DA55002000000000BA
S113C0E0000000000000000000000000000000004C
S113C0F00000000008ED00E01002010035B7000068
S113C10011020100E1BB0000270201007197000049
S113C1102803010021B100003E020100BDBF000060
S113C1208502010041BD00002203000091A200002D
S113C1302E04000045B300001404000081BE00007A
S113C1401903010049B500002F0300009DA500005C
S113C150310401002B9200003405000071A8000096
S113C16036020000B5AA00003701000081BA0000C1
S113C17072B6002100220023002400250026002797
S113C180B846B946BA46BB46BC460A490A4A521A98
S113C190013A05DD0020042308601944043AFBDA5F
S113C1A006488546064880470648804762B6F9F740
S113C1B025FFFEE700000020EF5B0020F05B00207D
S113C1C0059E000021C000000000010031070000AE
S113C1D00001080001000000FFFFFFFF0100010053
S113C1E0DF0700000001080001000000FFFFFFFF5F
S113C1F002000100B1070000000008000000000078
S113C200FFFFFFFF030001003402000000000800EC
S113C21000000000FFFFFFFF0300011302401D01A7
S113C2200B000600070008000C001C00180017048F
S113C2300E000F4004033D0121503E543F4C3C0589
S113C24023002400250026002700280029002A00B6
S113C2502C002D002E002F0030003100320033005E
S113C2602B0034000000000046697273742066726B
S113C270616D652073686F756C64206E6F742075D2
S113C2807365206D756C7469706C65206672616D80
S113C29065207472616E736D697373696F6E2E00BD
S113C2A04D756C74692D6672616D6520726573706D
S113C2B06F6E736520746F6F206C617267652066A2
S113C2C06F7220726563656976696E672062756650
S113C2D06665722E000000004D657373616765200A
S113C2E073697A6520746F6F206C617267652E20A4
S113C2F05365742061206C61726765722073656E8A
S113C30064206275666665720A00000041626F729D
S113C310742070726576696F7573206D65737361CF
S113C32067652C207472616E736D697373696F6EC7
S113C33020696E2070726F67726573732E0A000035
S113C34000000000000000000000000000000000E9
S113C35000000000000000000000000000000000D9
S113C36000000000000000000000000000000000C9
S113C37053696E676C652D6672616D65206C656EC0
S113C38067746820746F6F20736D616C6C206F72BA
S113C39020746F6F206C617267652E00466972733A
S113C3A074206672616D652073686F756C642062B9
S113C3B065203820627974657320696E206C656E1F
S113C3C06774682E00000000436F6E7365637574B4
S113C3D0697665206672616D6520746F6F2073687D
S113C3E06F72742E00000000466C6F7720636F6ECE
S113C3F074726F6C206672616D6520746F6F207348
S113C400686F72742E00000001000000020000003A
S113C41004000000080000001000000020000000DC
S113C420400000008000000000F00DF8002801D05A
S113C43000BF00BF00BF00BF002000BF00BFF9F76E
S113C440DDFD00F002F80120704780B500F002F82D
S113C45001BD00000746384600F002F8FBE7000083
S113C46080B500BF00BF024A11001820ABBEFBE735
S113C470260002000548014603B4684680F3098893
S113C48000BF00BF00BF00BFFFF7CEFFA5EDF5FE64
S113C4902D2D2D2D2D4A756D70546F4170702D2DDD
S113C4A02D2D2D0A000000002D2D2D2D2D494E542B
S113C4B04F20424F4F542D2D2D2D2D0A00000000EA
S113C4C025303464203A204D5F535F4354524C204E
S113C4D03D20307825780A00303132333435363710
S113C4E038394142434445465465726D696E616C06
S113C4F00000000053454747455200000102030471
S107C5004D535751EB
S903C475C3
